** EXPERIMENTAL (HLL) ** Open Watcom Linker Version 1.6beta1 Limited Availability
Portions Copyright (c) 1985-2002 Sybase, Inc. All Rights Reserved.
Created on:       13/11/17 16:25:11
Warning! W1121: file U:/tmp\ldconv__hashopenssl_obj_1a0352885a3d184530.obj(U:\DEV\python-2.7.5\Modules\_hashopenssl.c): '_init_hashlib' has already been exported
Executable Image: build/lib.os2knix-2.7/_hashlib.pyd
creating an OS/2 EMX dynamic link library


                        +------------+
                        |   Groups   |
                        +------------+

Group                           Address              Size
=====                           =======              ====

CGROUP                          0001:00000000        000e03f0
DGROUP                          0002:00000000        00003d30



                        +--------------+
                        |   Segments   |
                        +--------------+

Segment                Class          Group          Address         Size
=======                =====          =====          =======         ====

TEXT32                 CODE           CGROUP         0001:00000000   000e03f0
________TEXT           CODE           CGROUP         0001:000e03f0   00000000
DATA32                 DATA           DGROUP         0002:00000000   000016a0
SET1__os2dll           DATA           DGROUP         0002:000016a0   00000004
SET2__os2dll           DATA           DGROUP         0002:000016a4   00000000
SET3__os2dll           DATA           DGROUP         0002:000016a4   00000004
SET1___CTOR_LIST__     DATA           DGROUP         0002:000016a8   00000004
SET2___CTOR_LIST__     DATA           DGROUP         0002:000016ac   00000000
SET3___CTOR_LIST__     DATA           DGROUP         0002:000016ac   00000004
SET1___DTOR_LIST__     DATA           DGROUP         0002:000016b0   00000004
SET2___DTOR_LIST__     DATA           DGROUP         0002:000016b4   00000000
SET3___DTOR_LIST__     DATA           DGROUP         0002:000016b4   00000004
SET1___crtinit1__      DATA           DGROUP         0002:000016b8   00000004
SET2___crtinit1__      DATA           DGROUP         0002:000016bc   00000000
SET3___crtinit1__      DATA           DGROUP         0002:000016bc   00000004
SET1___crtexit1__      DATA           DGROUP         0002:000016c0   00000004
SET2___crtexit1__      DATA           DGROUP         0002:000016c4   00000000
SET3___crtexit1__      DATA           DGROUP         0002:000016c4   00000004
SET1___eh_frame__      DATA           DGROUP         0002:000016c8   00000004
SET2___eh_frame__      DATA           DGROUP         0002:000016cc   00000008
SET3___eh_frame__      DATA           DGROUP         0002:000016d4   00000004
SET1___eh_init__       DATA           DGROUP         0002:000016d8   00000004
SET2___eh_init__       DATA           DGROUP         0002:000016dc   00000004
SET3___eh_init__       DATA           DGROUP         0002:000016e0   00000004
SET1___eh_term__       DATA           DGROUP         0002:000016e4   00000004
SET2___eh_term__       DATA           DGROUP         0002:000016e8   00000004
SET3___eh_term__       DATA           DGROUP         0002:000016ec   00000004
SET1___fork_parent1__  DATA           DGROUP         0002:000016f0   00000004
SET2___fork_parent1__  DATA           DGROUP         0002:000016f4   00000000
SET3___fork_parent1__  DATA           DGROUP         0002:000016f4   00000004
SET1___fork_child1__   DATA           DGROUP         0002:000016f8   00000004
SET2___fork_child1__   DATA           DGROUP         0002:000016fc   00000000
SET3___fork_child1__   DATA           DGROUP         0002:000016fc   00000004
________DATA           DATA           DGROUP         0002:00001700   00000000
BSS32                  BSS            DGROUP         0002:00001700   00002610
c_common               BSS            DGROUP         0002:00003d10   00000020
________BSS            BSS            DGROUP         0002:00003d30   00000000


                        +----------------+
                        |   Memory Map   |
                        +----------------+

* = unreferenced symbol
+ = symbol only referenced locally

Address        Symbol
=======        ======

Module: U:\usr\lib\dll0hi.obj({standard input})
0001:00000000* __text
0002:00000000* __data
0002:00000000* ___data_start
0002:00001700* ___bss_start
0002:000016a0+ __os2dll
0002:000016a8  ___CTOR_LIST__
0002:000016b0  ___DTOR_LIST__
0002:000016b8* ___crtinit1__
0002:000016c0* ___crtexit1__
0002:000016c8  ___eh_frame__
0002:000016d8  ___eh_init__
0002:000016e4  ___eh_term__
0002:000016f0+ ___fork_parent1__
0002:000016f8+ ___fork_child1__
Module: U:/tmp\ldconv__hashopenssl_obj_1a0352885a3d184530.obj(U:\DEV\python-2.7.5\Modules\_hashopenssl.c)
0001:00000ad9  _init_hashlib
Module: U:\usr\local473\lib\libc_dll.lib(dllinit.obj)
0001:00000fb0  _DLL_InitTerm
Module: U:\usr\lib\libend.lib(src/libend/386/endlink386.asm)
0002:00003d30  _end
0002:00001700  _edata
Module: U:\usr\lib\libend.lib(src/libend/386/end.asm)
0001:000e03f0* _etext
0001:000e03f0* __etext
0000:00000000  WEAK$ZERO
0002:00003d30  __end
0002:00001700  __edata
Module: U:\extras\lib\libcrypto.lib(evp_lib.obj)
0001:00001010  _EVP_CIPHER_param_to_asn1
0001:0000104a  _EVP_CIPHER_asn1_to_param
0001:000010a1* _EVP_CIPHER_get_asn1_iv
0001:0000138b  _EVP_CIPHER_CTX_iv_length
0001:00001153* _EVP_CIPHER_set_asn1_iv
0001:000011ba  _EVP_CIPHER_type
0001:000013ae  _EVP_CIPHER_nid
0001:00001300* _EVP_CIPHER_block_size
0001:0000130b  _EVP_CIPHER_CTX_block_size
0001:00001318* _EVP_Cipher
0001:00001345  _EVP_CIPHER_CTX_cipher
0001:0000134f* _EVP_CIPHER_flags
0001:0000135a  _EVP_CIPHER_CTX_flags
0001:00001367* _EVP_CIPHER_CTX_get_app_data
0001:00001372* _EVP_CIPHER_CTX_set_app_data
0001:00001380  _EVP_CIPHER_iv_length
0001:00001398  _EVP_CIPHER_key_length
0001:000013a3  _EVP_CIPHER_CTX_key_length
0001:000013b8* _EVP_CIPHER_CTX_nid
0001:000013c4  _EVP_MD_block_size
0001:000013cf  _EVP_MD_type
0001:000013d9  _EVP_MD_pkey_type
0001:000013e4  _EVP_MD_size
0001:0000142b* _EVP_MD_flags
0001:00001436  _EVP_MD_CTX_md
0001:0000144d  _EVP_MD_CTX_set_flags
0001:00001463  _EVP_MD_CTX_clear_flags
0001:0000147b  _EVP_MD_CTX_test_flags
0001:0000148b* _EVP_CIPHER_CTX_set_flags
0001:000014a1* _EVP_CIPHER_CTX_clear_flags
0001:000014b9* _EVP_CIPHER_CTX_test_flags
Module: U:\extras\lib\libcrypto.lib(digest.obj)
0001:000014d0  _EVP_MD_CTX_init
0001:000014fc  _EVP_MD_CTX_create
0001:00001537  _EVP_DigestInit
0001:00001564  _EVP_DigestInit_ex
0001:0000182d  _EVP_DigestUpdate
0001:00001851  _EVP_DigestFinal
0001:000018ac  _EVP_DigestFinal_ex
0001:00001c61  _EVP_MD_CTX_cleanup
0001:00001962  _EVP_MD_CTX_copy
0001:00001987  _EVP_MD_CTX_copy_ex
0001:00001ba9  _EVP_Digest
0001:00001c43  _EVP_MD_CTX_destroy
Module: U:\extras\lib\libcrypto.lib(names.obj)
0001:00001d60* _EVP_add_cipher
0001:00001dd8  _EVP_add_digest
0001:00001eed  _EVP_get_cipherbyname
0001:00001f0e  _EVP_get_digestbyname
0001:00001f2f* _EVP_cleanup
0001:00001ff5* _EVP_CIPHER_do_all
0001:00002024* _EVP_CIPHER_do_all_sorted
0001:000020ca* _EVP_MD_do_all
0001:000020f9* _EVP_MD_do_all_sorted
Module: U:\extras\lib\libcrypto.lib(c_alld.obj)
0001:000021a1  _OpenSSL_add_all_digests
Module: U:\tmp\ldconv_libgcc_so_d_a_1a0352885a3e1639c0.lib(emx-ctordtor.obj)
0001:00002360  ___ctordtorInit
0001:00002394  ___ctordtorTerm
Module: U:\extras\lib\libcrypto.lib(cryptlib.obj)
0001:000025bf* _CRYPTO_get_new_lockid
0001:0000268e* _CRYPTO_num_locks
0001:00002698* _CRYPTO_get_new_dynlockid
0001:00002d5d  _CRYPTO_lock
0001:0000294d* _CRYPTO_destroy_dynlockid
0001:00002a8b* _CRYPTO_get_dynlock_value
0001:00002b43* _CRYPTO_get_dynlock_create_callback
0001:00002b4d* _CRYPTO_get_dynlock_lock_callback
0001:00002b57* _CRYPTO_get_dynlock_destroy_callback
0001:00002b61* _CRYPTO_set_dynlock_create_callback
0001:00002b6e* _CRYPTO_set_dynlock_lock_callback
0001:00002b7b* _CRYPTO_set_dynlock_destroy_callback
0001:00002b88* _CRYPTO_get_locking_callback
0001:00002b92* _CRYPTO_get_add_lock_callback
0001:00002b9c* _CRYPTO_set_locking_callback
0001:00002ba9* _CRYPTO_set_add_lock_callback
0001:00002bb6* _CRYPTO_THREADID_set_numeric
0001:00002bea* _CRYPTO_THREADID_set_pointer
0001:00002c36* _CRYPTO_THREADID_set_callback
0001:00002c58* _CRYPTO_THREADID_get_callback
0001:00002c62  _CRYPTO_THREADID_current
0001:00002cb8  _CRYPTO_THREADID_cmp
0001:00002cda  _CRYPTO_THREADID_cpy
0001:00002cfc  _CRYPTO_THREADID_hash
0001:00002d07* _CRYPTO_get_id_callback
0001:00002d11* _CRYPTO_set_id_callback
0001:00002d1e* _CRYPTO_thread_id
0001:00002f8a  _OpenSSLDie
0001:00002e04  _CRYPTO_add_lock
0001:00002eb1* _CRYPTO_get_lock_name
0001:00002f12* _OPENSSL_ia32cap_loc
0001:00002f1c* _OPENSSL_cpuid_setup
0001:00002f21* _OPENSSL_showfatal
0001:00002f4a* _OPENSSL_isservice
0001:00002fb6* _OPENSSL_stderr
0002:00001890* _OPENSSL_ia32cap_P
0002:00001894* _OPENSSL_NONPIC_relocated
Module: U:\extras\lib\libcrypto.lib(evp_asn1.obj)
0001:00002fc0  _ASN1_TYPE_set_octetstring
0001:00003032  _ASN1_TYPE_get_octetstring
0001:000030ca* _ASN1_TYPE_set_int_octetstring
0001:00003237* _ASN1_TYPE_get_int_octetstring
Module: U:\extras\lib\libcrypto.lib(obj_dat.obj)
0001:0001256f  _OBJ_bsearch_
0001:000117d1  _check_defer
0001:000117f2  _OBJ_cleanup
0001:0001187d* _OBJ_new_nid
0001:000118a7* _OBJ_add_object
0001:00011abf  _OBJ_nid2obj
0001:00011bb4  _OBJ_nid2sn
0001:00011cac  _OBJ_nid2ln
0001:00011e66  _OBJ_obj2nid
0001:00011f0e  _OBJ_txt2obj
0001:000124de  _OBJ_sn2nid
0001:0001244d  _OBJ_ln2nid
0001:0001206b  _OBJ_obj2txt
0001:00012413* _OBJ_txt2nid
0001:000125a6  _OBJ_bsearch_ex_
0001:000126a8* _OBJ_create_objects
0001:00012875* _OBJ_create
0002:00001930  _obj_cleanup_defer
Module: U:\extras\lib\libcrypto.lib(a_object.obj)
0001:000129b0* _i2d_ASN1_OBJECT
0001:00012a79  _a2d_ASN1_OBJECT
0001:00012f10  _i2t_ASN1_OBJECT
0001:00012f48  _i2a_ASN1_OBJECT
0001:00013043  _d2i_ASN1_OBJECT
0001:00013109  _c2i_ASN1_OBJECT
0001:00013312  _ASN1_OBJECT_new
0001:000133b0  _ASN1_OBJECT_free
0001:00013466  _ASN1_OBJECT_create
Module: U:\extras\lib\libcrypto.lib(err.obj)
0001:00013991* _ERR_get_implementation
0001:000139a3* _ERR_set_implementation
0001:000143f6* _ERR_load_ERR_strings
0001:0001449d* _ERR_load_strings
0001:000144bc* _ERR_unload_strings
0001:00014501* _ERR_free_strings
0001:00014518  _ERR_put_error
0001:00014f83* _ERR_get_state
0001:00014675  _ERR_clear_error
0001:0001475a* _ERR_get_error
0001:00014796* _ERR_get_error_line
0001:000147d0  _ERR_get_error_line_data
0001:00014808  _ERR_peek_error
0001:00014844* _ERR_peek_error_line
0001:0001487e* _ERR_peek_error_line_data
0001:000148b6  _ERR_peek_last_error
0001:000148f2* _ERR_peek_last_error_line
0001:0001492c* _ERR_peek_last_error_line_data
0001:00014bae  _ERR_error_string_n
0001:00014de4* _ERR_lib_error_string
0001:00014e2e* _ERR_func_error_string
0001:00014e95* _ERR_reason_error_string
0001:00014d5a* _ERR_error_string
0001:00014d8c* _ERR_get_string_table
0001:00014da9* _ERR_get_err_state_table
0001:00014dc7* _ERR_release_err_state_table
0001:00014f21* _ERR_remove_thread_state
0001:00014f6f* _ERR_remove_state
0001:000150c0* _ERR_get_next_error_library
0001:000150d7* _ERR_set_error_data
0001:0001517c  _ERR_add_error_data
0001:00015289  _ERR_set_mark
0001:000152e0  _ERR_pop_to_mark
Module: U:\extras\lib\libcrypto.lib(mem.obj)
0001:000154b9* _CRYPTO_set_mem_functions
0001:00015532* _CRYPTO_set_mem_ex_functions
0001:000155ab* _CRYPTO_set_locked_mem_functions
0001:000155f2* _CRYPTO_set_locked_mem_ex_functions
0001:00015639* _CRYPTO_set_mem_debug_functions
0001:0001567b* _CRYPTO_get_mem_functions
0001:000156d7* _CRYPTO_get_mem_ex_functions
0001:00015733* _CRYPTO_get_locked_mem_functions
0001:0001576c* _CRYPTO_get_locked_mem_ex_functions
0001:000157a5* _CRYPTO_get_mem_debug_functions
0001:000157ff  _CRYPTO_malloc_locked
0001:000158d7  _CRYPTO_free_locked
0001:0001592b  _CRYPTO_malloc
0001:00015a03* _CRYPTO_strdup
0001:00015a45  _CRYPTO_realloc
0001:00015b28  _CRYPTO_realloc_clean
0001:00015c43  _CRYPTO_free
0001:00015c9d* _CRYPTO_remalloc
0001:00015cd7* _CRYPTO_set_mem_debug_options
0001:00015cf6* _CRYPTO_get_mem_debug_options
Module: U:\extras\lib\libcrypto.lib(eng_init.obj)
0001:00015d20  _engine_unlocked_init
0001:00015d86  _engine_unlocked_finish
0001:00015e77  _ENGINE_init
0001:00015f11  _ENGINE_finish
Module: U:\extras\lib\libcrypto.lib(tb_digest.obj)
0001:00016000* _ENGINE_unregister_digests
0001:0001602f* _ENGINE_register_digests
0001:000160a7* _ENGINE_register_all_digests
0001:000160d8* _ENGINE_set_default_digests
0001:00016150  _ENGINE_get_digest_engine
0001:00016177  _ENGINE_get_digest
0001:000161ee* _ENGINE_get_digests
0001:000161f9* _ENGINE_set_digests
Module: U:\extras\lib\libcrypto.lib(pmeth_lib.obj)
0001:00016280* _EVP_PKEY_meth_find
0001:000168eb  _EVP_PKEY_CTX_free
0001:00016537* _EVP_PKEY_meth_new
0001:00016681  _EVP_PKEY_meth_free
0001:000166a7  _EVP_PKEY_CTX_new
0001:000166c9  _EVP_PKEY_CTX_new_id
0001:000166eb  _EVP_PKEY_CTX_dup
0001:00016887* _EVP_PKEY_meth_add0
0001:00016974  _EVP_PKEY_CTX_ctrl
0001:00016ad3* _EVP_PKEY_CTX_ctrl_str
0001:00016be6* _EVP_PKEY_CTX_get_operation
0001:00016bf1* _EVP_PKEY_CTX_set0_keygen_info
0001:00016c08* _EVP_PKEY_CTX_set_data
0001:00016c16* _EVP_PKEY_CTX_get_data
0001:00016c21* _EVP_PKEY_CTX_get0_pkey
0001:00016c2c* _EVP_PKEY_CTX_get0_peerkey
0001:00016c37* _EVP_PKEY_CTX_set_app_data
0001:00016c45* _EVP_PKEY_CTX_get_app_data
0001:00016c50* _EVP_PKEY_meth_set_init
0001:00016c5e* _EVP_PKEY_meth_set_copy
0001:00016c6c* _EVP_PKEY_meth_set_cleanup
0001:00016c7a* _EVP_PKEY_meth_set_paramgen
0001:00016c91* _EVP_PKEY_meth_set_keygen
0001:00016ca8* _EVP_PKEY_meth_set_sign
0001:00016cbf* _EVP_PKEY_meth_set_verify
0001:00016cd6* _EVP_PKEY_meth_set_verify_recover
0001:00016ced* _EVP_PKEY_meth_set_signctx
0001:00016d04* _EVP_PKEY_meth_set_verifyctx
0001:00016d1b* _EVP_PKEY_meth_set_encrypt
0001:00016d32* _EVP_PKEY_meth_set_decrypt
0001:00016d49* _EVP_PKEY_meth_set_derive
0001:00016d60* _EVP_PKEY_meth_set_ctrl
0002:00003060* _app_pkey_methods
Module: U:\extras\lib\libcrypto.lib(mem_clr.obj)
0001:00016d80  _OPENSSL_cleanse
0002:00003070  _cleanse_ctr
Module: U:\extras\lib\libcrypto.lib(o_names.obj)
0001:00016e4f* _OBJ_NAME_init
0001:00016eaf* _OBJ_NAME_new_index
0001:0001713e  _OBJ_NAME_get
0001:000171e9  _OBJ_NAME_add
0001:0001730e* _OBJ_NAME_remove
0001:0001741f  _OBJ_NAME_do_all
0001:000174c6  _OBJ_NAME_do_all_sorted
0001:000175ea  _OBJ_NAME_cleanup
Module: U:\extras\lib\libcrypto.lib(evp_pbe.obj)
0001:00017825  _EVP_PBE_CipherInit
0001:00017c46  _EVP_PBE_find
0001:00017b1c* _EVP_PBE_alg_add_type
0001:00017bdc* _EVP_PBE_alg_add
0001:00017d2a  _EVP_PBE_cleanup
Module: U:\extras\lib\libcrypto.lib(obj_xref.obj)
0002:00003d10+ _sig_app
0002:00003d20+ _sigx_app
0001:00018052  _OBJ_find_sigid_algs
0001:000180f0  _OBJ_find_sigid_by_algs
0001:000181a1* _OBJ_add_sigid
0001:000182c9  _OBJ_sigid_free
Module: U:\extras\lib\libcrypto.lib(m_md4.obj)
0001:000183cc  _EVP_md4
Module: U:\extras\lib\libcrypto.lib(m_md5.obj)
0001:0001848c  _EVP_md5
Module: U:\extras\lib\libcrypto.lib(m_sha.obj)
0001:0001854c  _EVP_sha
Module: U:\extras\lib\libcrypto.lib(m_dss.obj)
0001:0001860c  _EVP_dss
Module: U:\extras\lib\libcrypto.lib(m_sha1.obj)
0001:000186cc  _EVP_sha1
0001:0001879c  _EVP_sha224
0001:000187fc  _EVP_sha256
0001:000188cc  _EVP_sha384
0001:0001892c  _EVP_sha512
Module: U:\extras\lib\libcrypto.lib(m_dss1.obj)
0001:000189ec  _EVP_dss1
Module: U:\extras\lib\libcrypto.lib(m_ecdsa.obj)
0001:00018aac  _EVP_ecdsa
Module: U:\extras\lib\libcrypto.lib(m_mdc2.obj)
0001:00018b6c  _EVP_mdc2
Module: U:\extras\lib\libcrypto.lib(m_ripemd.obj)
0001:00018c2c  _EVP_ripemd160
Module: U:\extras\lib\libcrypto.lib(m_wp.obj)
0001:00018cec  _EVP_whirlpool
Module: U:\tmp\ldconv_libgcc_so_d_a_1a0352885a3e1639c0.lib(emx-eh.obj)
0001:00018d00  ___ehInit
0001:00018d36* ___ehTerm
Module: U:\extras\lib\libcrypto.lib(stack.obj)
0001:00018d70* _STACK_version
0001:00018d99  _sk_set_cmp_func
0001:00018dd3  _sk_dup
0001:00018ec0  _sk_new
0001:000193f6  _sk_free
0001:00018eac  _sk_new_null
0001:00018f86  _sk_insert
0001:0001909f  _sk_delete_ptr
0001:000190eb  _sk_delete
0001:000194aa  _sk_sort
0001:00019251  _sk_find
0001:00019273* _sk_find_ex
0001:00019295  _sk_push
0001:000192b8* _sk_unshift
0001:000192da* _sk_shift
0001:00019312  _sk_pop
0001:0001934c* _sk_zero
0001:00019398  _sk_pop_free
0001:0001942a  _sk_num
0001:00019441  _sk_value
0001:00019473  _sk_set
0001:000194fd  _sk_is_sorted
Module: U:\extras\lib\libcrypto.lib(buffer.obj)
0001:00019529  _BUF_MEM_new
0001:000195a9  _BUF_MEM_free
0001:000195fd  _BUF_MEM_grow
0001:00019759  _BUF_MEM_grow_clean
0001:000198e8  _BUF_strdup
0001:00019917* _BUF_strndup
0001:00019a26  _BUF_strlcpy
0001:000199a1* _BUF_memdup
0001:00019a76  _BUF_strlcat
0001:00019abb* _BUF_reverse
Module: U:\extras\lib\libcrypto.lib(asn1_lib.obj)
0001:00019b40* _ASN1_version
0001:00019bb1* _ASN1_check_infinite_end
0001:00019bcb  _ASN1_const_check_infinite_end
0001:00019bf0  _ASN1_get_object
0001:00019eb2  _ASN1_put_object
0001:00019fb2  _ASN1_put_eoc
0001:0001a065  _ASN1_object_size
0001:0001a13f* _asn1_Finish
0001:0001a152  _asn1_const_Finish
0001:0001a165  _asn1_GetSequence
0001:0001a26a  _ASN1_STRING_copy
0001:0001a31a  _ASN1_STRING_set
0001:0001a2c5  _ASN1_STRING_dup
0001:0001a479  _ASN1_STRING_new
0001:0001a516  _ASN1_STRING_free
0001:0001a448  _ASN1_STRING_set0
0001:0001a48d  _ASN1_STRING_type_new
0001:0001a557  _ASN1_STRING_cmp
0001:0001a5d9  _asn1_add_error
0001:0001a64f* _ASN1_STRING_length
0001:0001a659* _ASN1_STRING_length_set
0001:0001a666* _ASN1_STRING_type
0001:0001a671  _ASN1_STRING_data
Module: U:\extras\lib\libcrypto.lib(a_type.obj)
0001:0001a680  _ASN1_TYPE_get
0001:0001a6a5  _ASN1_TYPE_set
0001:0001a701  _ASN1_TYPE_set1
0001:0001a7ab  _ASN1_TYPE_cmp
Module: U:\extras\lib\libcrypto.lib(a_int.obj)
0001:0001a830* _ASN1_INTEGER_dup
0001:0001a843  _ASN1_INTEGER_cmp
0001:0001a8a2  _i2c_ASN1_INTEGER
0001:0001aa74  _c2i_ASN1_INTEGER
0001:0001aca6  _d2i_ASN1_UINTEGER
0001:0001ae72  _ASN1_INTEGER_set
0001:0001afae  _ASN1_INTEGER_get
0001:0001b058  _BN_to_ASN1_INTEGER
0001:0001b1c9  _ASN1_INTEGER_to_BN
Module: U:\extras\lib\libcrypto.lib(tasn_typ.obj)
0001:0001b260  _ASN1_INTEGER_it
0001:0001b27c  _d2i_ASN1_INTEGER
0001:0001b2a5  _i2d_ASN1_INTEGER
0001:0001b2c7  _ASN1_INTEGER_new
0001:0001b2db  _ASN1_INTEGER_free
0001:0001b310  _ASN1_ENUMERATED_it
0001:0001b32c  _d2i_ASN1_ENUMERATED
0001:0001b355* _i2d_ASN1_ENUMERATED
0001:0001b377* _ASN1_ENUMERATED_new
0001:0001b38b  _ASN1_ENUMERATED_free
0001:0001b3c0  _ASN1_BIT_STRING_it
0001:0001b3dc  _d2i_ASN1_BIT_STRING
0001:0001b405  _i2d_ASN1_BIT_STRING
0001:0001b427  _ASN1_BIT_STRING_new
0001:0001b43b  _ASN1_BIT_STRING_free
0001:0001b470  _ASN1_OCTET_STRING_it
0001:0001b48c  _d2i_ASN1_OCTET_STRING
0001:0001b4b5  _i2d_ASN1_OCTET_STRING
0001:0001b4d7  _ASN1_OCTET_STRING_new
0001:0001b4eb  _ASN1_OCTET_STRING_free
0001:0001b510  _ASN1_NULL_it
0001:0001b52c* _d2i_ASN1_NULL
0001:0001b555* _i2d_ASN1_NULL
0001:0001b577  _ASN1_NULL_new
0001:0001b58b* _ASN1_NULL_free
0001:0001b5c0  _ASN1_OBJECT_it
0001:0001b5f0  _ASN1_UTF8STRING_it
0001:0001b60c* _d2i_ASN1_UTF8STRING
0001:0001b635* _i2d_ASN1_UTF8STRING
0001:0001b657  _ASN1_UTF8STRING_new
0001:0001b66b  _ASN1_UTF8STRING_free
0001:0001b6a0* _ASN1_PRINTABLESTRING_it
0001:0001b6bc* _d2i_ASN1_PRINTABLESTRING
0001:0001b6e5* _i2d_ASN1_PRINTABLESTRING
0001:0001b707* _ASN1_PRINTABLESTRING_new
0001:0001b71b* _ASN1_PRINTABLESTRING_free
0001:0001b750* _ASN1_T61STRING_it
0001:0001b76c* _d2i_ASN1_T61STRING
0001:0001b795* _i2d_ASN1_T61STRING
0001:0001b7b7* _ASN1_T61STRING_new
0001:0001b7cb* _ASN1_T61STRING_free
0001:0001b800  _ASN1_IA5STRING_it
0001:0001b81c* _d2i_ASN1_IA5STRING
0001:0001b845* _i2d_ASN1_IA5STRING
0001:0001b867* _ASN1_IA5STRING_new
0001:0001b87b* _ASN1_IA5STRING_free
0001:0001b8b0* _ASN1_GENERALSTRING_it
0001:0001b8cc* _d2i_ASN1_GENERALSTRING
0001:0001b8f5* _i2d_ASN1_GENERALSTRING
0001:0001b917* _ASN1_GENERALSTRING_new
0001:0001b92b* _ASN1_GENERALSTRING_free
0001:0001b960* _ASN1_UTCTIME_it
0001:0001b97c* _d2i_ASN1_UTCTIME
0001:0001b9a5* _i2d_ASN1_UTCTIME
0001:0001b9c7* _ASN1_UTCTIME_new
0001:0001b9db* _ASN1_UTCTIME_free
0001:0001ba10  _ASN1_GENERALIZEDTIME_it
0001:0001ba2c* _d2i_ASN1_GENERALIZEDTIME
0001:0001ba55* _i2d_ASN1_GENERALIZEDTIME
0001:0001ba77  _ASN1_GENERALIZEDTIME_new
0001:0001ba8b* _ASN1_GENERALIZEDTIME_free
0001:0001bac0* _ASN1_VISIBLESTRING_it
0001:0001badc* _d2i_ASN1_VISIBLESTRING
0001:0001bb05* _i2d_ASN1_VISIBLESTRING
0001:0001bb27* _ASN1_VISIBLESTRING_new
0001:0001bb3b* _ASN1_VISIBLESTRING_free
0001:0001bb70* _ASN1_UNIVERSALSTRING_it
0001:0001bb8c* _d2i_ASN1_UNIVERSALSTRING
0001:0001bbb5* _i2d_ASN1_UNIVERSALSTRING
0001:0001bbd7* _ASN1_UNIVERSALSTRING_new
0001:0001bbeb* _ASN1_UNIVERSALSTRING_free
0001:0001bc20* _ASN1_BMPSTRING_it
0001:0001bc3c* _d2i_ASN1_BMPSTRING
0001:0001bc65* _i2d_ASN1_BMPSTRING
0001:0001bc87* _ASN1_BMPSTRING_new
0001:0001bc9b* _ASN1_BMPSTRING_free
0001:0001bcc0  _ASN1_ANY_it
0001:0001bcf0  _ASN1_SEQUENCE_it
0001:0001bd0c  _d2i_ASN1_TYPE
0001:0001bd35  _i2d_ASN1_TYPE
0001:0001bd57  _ASN1_TYPE_new
0001:0001bd6b  _ASN1_TYPE_free
0001:0001bda0  _ASN1_PRINTABLE_it
0001:0001bdbc* _d2i_ASN1_PRINTABLE
0001:0001bde5* _i2d_ASN1_PRINTABLE
0001:0001be07* _ASN1_PRINTABLE_new
0001:0001be1b* _ASN1_PRINTABLE_free
0001:0001be50  _DISPLAYTEXT_it
0001:0001be6c* _d2i_DISPLAYTEXT
0001:0001be95* _i2d_DISPLAYTEXT
0001:0001beb7* _DISPLAYTEXT_new
0001:0001becb* _DISPLAYTEXT_free
0001:0001bf00  _DIRECTORYSTRING_it
0001:0001bf1c* _d2i_DIRECTORYSTRING
0001:0001bf45* _i2d_DIRECTORYSTRING
0001:0001bf67* _DIRECTORYSTRING_new
0001:0001bf7b* _DIRECTORYSTRING_free
0001:0001bfb0  _ASN1_BOOLEAN_it
0001:0001bfe0* _ASN1_TBOOLEAN_it
0001:0001c010  _ASN1_FBOOLEAN_it
0001:0001c050  _ASN1_OCTET_STRING_NDEF_it
0001:0001c0a0* _ASN1_SEQUENCE_ANY_it
0001:0001c0f0* _ASN1_SET_ANY_it
0001:0001c10c  _d2i_ASN1_SEQUENCE_ANY
0001:0001c135  _i2d_ASN1_SEQUENCE_ANY
0001:0001c157* _d2i_ASN1_SET_ANY
0001:0001c180  _i2d_ASN1_SET_ANY
Module: U:\extras\lib\libcrypto.lib(a_bytes.obj)
0001:0001c1ba* _d2i_ASN1_type_bytes
0001:0001c3ae  _i2d_ASN1_bytes
0001:0001c49a* _d2i_ASN1_bytes
Module: U:\extras\lib\libcrypto.lib(lhash.obj)
0001:0001c920* _lh_version
0001:0001c951  _lh_new
0001:0001d28b  _lh_strhash
0001:0001caee  _lh_free
0001:0001cb62  _lh_insert
0001:0001cc80  _lh_delete
0001:0001cd5a  _lh_retrieve
0001:0001ce3b  _lh_doall
0001:0001ce6d  _lh_doall_arg
0001:0001d302  _lh_num_items
Module: U:\extras\lib\libcrypto.lib(obj_lib.obj)
0001:0001d32a  _OBJ_dup
0001:0001d597  _OBJ_cmp
Module: U:\extras\lib\libcrypto.lib(bn_word.obj)
0001:0001d5f0  _BN_mod_word
0001:0001d674  _BN_div_word
0001:0001d794  _BN_add_word
0001:0001d8ec  _BN_sub_word
0001:0001da66  _BN_mul_word
Module: U:\extras\lib\libcrypto.lib(bn_lib.obj)
0001:0001db40* _BN_version
0001:0001db6e* _BN_set_params
0001:0001dc35* _BN_get_params
0001:0001dc73  _BN_value_one
0001:0001dc87* _BN_options
0001:0001dcd4  _BN_num_bits_word
0001:0001dd45  _BN_num_bits
0001:0001dd8f  _BN_clear_free
0001:0001de11  _BN_free
0001:0001de79  _BN_init
0001:0001dea5  _BN_new
0001:0001e0f7* _bn_dup_expand
0001:0001e1e2  _BN_dup
0001:0001e183  _bn_expand2
0001:0001e237  _BN_copy
0001:0001e370* _BN_swap
0001:0001e42a  _BN_clear
0001:0001e475* _BN_get_word
0001:0001e4a5  _BN_set_word
0001:0001e50c  _BN_bin2bn
0001:0001e67b  _BN_bn2bin
0001:0001e702  _BN_ucmp
0001:0001e78e  _BN_cmp
0001:0001e8a4  _BN_set_bit
0001:0001e99c* _BN_clear_bit
0001:0001ea71  _BN_is_bit_set
0001:0001eade  _BN_mask_bits
0001:0001ebd3  _BN_set_negative
0001:0001ebfe  _bn_cmp_words
0001:0001ec95  _bn_cmp_part_words
Module: U:\extras\lib\libcrypto.lib(bn_shift.obj)
0001:0001ee50  _BN_lshift1
0001:0001ef6a  _BN_rshift1
0001:0001f0ab  _BN_lshift
0001:0001f290  _BN_rshift
Module: U:\extras\lib\libcrypto.lib(bn_print.obj)
0001:0001f4fc* _BN_bn2hex
0001:0001f630  _BN_bn2dec
0001:0001f8b3  _BN_hex2bn
0001:0001fb28  _BN_dec2bn
0001:0001fd5a  _BN_asc2bn
0001:0001fde9* _BN_print_fp
0001:0001fe57* _BN_print
Module: U:\extras\lib\libcrypto.lib(b_print.obj)
0001:000213a4  _BIO_printf
0001:000213d9* _BIO_vprintf
0001:000214cd  _BIO_snprintf
0001:00021501* _BIO_vsnprintf
Module: U:\extras\lib\libcrypto.lib(bio_lib.obj)
0001:0002157a  _BIO_new
0001:0002160c  _BIO_set
0001:00021700  _BIO_free
0001:00021800  _BIO_vfree
0001:00021813  _BIO_clear_flags
0001:0002182b  _BIO_test_flags
0001:00021839  _BIO_set_flags
0001:0002184f* _BIO_get_callback
0001:0002185a* _BIO_set_callback
0001:00021868* _BIO_set_callback_arg
0001:00021876* _BIO_get_callback_arg
0001:00021881* _BIO_method_name
0001:0002188e* _BIO_method_type
0001:0002189a  _BIO_read
0001:000219f5  _BIO_write
0001:00021b5a  _BIO_puts
0001:00021cb0  _BIO_gets
0001:00021df6  _BIO_indent
0001:00021e4e  _BIO_int_ctrl
0001:00021eb9  _BIO_ctrl
0001:00021e7c* _BIO_ptr_ctrl
0001:00021fcc  _BIO_callback_ctrl
0001:000220da* _BIO_ctrl_pending
0001:00022105* _BIO_ctrl_wpending
0001:00022130  _BIO_push
0001:0002219b  _BIO_pop
0001:00022224* _BIO_get_retry_BIO
0001:0002227e* _BIO_get_retry_reason
0001:00022289  _BIO_find_type
0001:000222f4  _BIO_next
0001:0002230c  _BIO_free_all
0001:00022348* _BIO_dup_chain
0001:00022480  _BIO_copy_next_retry
0001:000224bc* _BIO_get_ex_new_index
0001:000224f3* _BIO_set_ex_data
0001:00022517* _BIO_get_ex_data
0001:00022534* _BIO_number_read
0001:0002254c* _BIO_number_written
Module: U:\extras\lib\libcrypto.lib(mem_dbg.obj)
0001:000225be  _CRYPTO_mem_ctrl
0001:000227a9* _CRYPTO_is_mem_check_on
0001:00022850* _CRYPTO_dbg_set_options
0001:0002285d* _CRYPTO_dbg_get_options
0001:00022ac2  _CRYPTO_push_info_
0001:00022bc9  _CRYPTO_pop_info
0001:00022c0c* _CRYPTO_remove_all_info
0001:00022c4d* _CRYPTO_dbg_malloc
0001:00022e7b* _CRYPTO_dbg_free
0001:00022f03* _CRYPTO_dbg_realloc
0001:00023423* _CRYPTO_mem_leaks
0001:00023575* _CRYPTO_mem_leaks_fp
0001:00023660* _CRYPTO_mem_leaks_cb
Module: U:\extras\lib\libcrypto.lib(eng_lib.obj)
0001:000236ea  _ENGINE_new
0001:0002378f* _engine_set_all_null
0001:0002383d  _engine_free_util
0001:0002393a  _ENGINE_free
0001:000239d0  _engine_cleanup_add_first
0001:00023a1b  _engine_cleanup_add_last
0001:00023a78* _ENGINE_cleanup
0001:00023abc* _ENGINE_get_ex_new_index
0001:00023af3* _ENGINE_set_ex_data
0001:00023b17* _ENGINE_get_ex_data
0001:00023b34* _ENGINE_set_id
0001:00023b82* _ENGINE_set_name
0001:00023bd1* _ENGINE_set_destroy_function
0001:00023be4* _ENGINE_set_init_function
0001:00023bf7* _ENGINE_set_finish_function
0001:00023c0a* _ENGINE_set_ctrl_function
0001:00023c1d* _ENGINE_set_flags
0001:00023c30* _ENGINE_set_cmd_defns
0001:00023c43* _ENGINE_get_id
0001:00023c4d* _ENGINE_get_name
0001:00023c58* _ENGINE_get_destroy_function
0001:00023c63* _ENGINE_get_init_function
0001:00023c6e* _ENGINE_get_finish_function
0001:00023c79* _ENGINE_get_ctrl_function
0001:00023c84* _ENGINE_get_flags
0001:00023c8f* _ENGINE_get_cmd_defns
0001:00023c9a* _ENGINE_get_static_state
Module: U:\extras\lib\libcrypto.lib(eng_table.obj)
0001:00023cb0* _ENGINE_get_table_flags
0001:00023cba* _ENGINE_set_table_flags
0001:00023d87  _engine_table_register
0001:00024048  _engine_table_unregister
0001:00024125  _engine_table_cleanup
0001:000241a9  _engine_table_select
0001:000243cb  _engine_table_doall
Module: U:\extras\lib\libcrypto.lib(eng_list.obj)
0001:00024a72* _ENGINE_remove
0001:00024703  _ENGINE_get_first
0001:00024773* _ENGINE_get_last
0001:000247e3  _ENGINE_get_next
0001:0002489f* _ENGINE_get_prev
0001:0002495b* _ENGINE_add
0001:00024c88* _ENGINE_by_id
0001:00024ef3* _ENGINE_up_ref
Module: U:\extras\lib\libcrypto.lib(rsa_pmeth.obj)
0001:00026040  _rsa_pkey_meth
Module: U:\extras\lib\libcrypto.lib(dh_pmeth.obj)
0001:000264f0  _dh_pkey_meth
Module: U:\extras\lib\libcrypto.lib(dsa_pmeth.obj)
0001:00026c70  _dsa_pkey_meth
Module: U:\extras\lib\libcrypto.lib(ec_pmeth.obj)
0001:000273f0  _ec_pkey_meth
Module: U:\extras\lib\libcrypto.lib(hm_pmeth.obj)
0001:00027900  _hmac_pkey_meth
Module: U:\extras\lib\libcrypto.lib(tb_pkmeth.obj)
0001:00027970* _ENGINE_unregister_pkey_meths
0001:0002799f* _ENGINE_register_pkey_meths
0001:00027a17* _ENGINE_register_all_pkey_meths
0001:00027a48* _ENGINE_set_default_pkey_meths
0001:00027ac0  _ENGINE_get_pkey_meth_engine
0001:00027ae7  _ENGINE_get_pkey_meth
0001:00027b5e* _ENGINE_get_pkey_meths
0001:00027b69* _ENGINE_set_pkey_meths
0001:00027b7c  _engine_pkey_meths_free
Module: U:\extras\lib\libcrypto.lib(p_lib.obj)
0001:00027c10* _EVP_PKEY_bits
0001:00027c4d  _EVP_PKEY_size
0001:00027c8a* _EVP_PKEY_save_parameters
0001:00027cef  _EVP_PKEY_copy_parameters
0001:00027da6  _EVP_PKEY_missing_parameters
0001:00027ddd  _EVP_PKEY_cmp_parameters
0001:00027e30  _EVP_PKEY_cmp
0001:00027eb6  _EVP_PKEY_new
0001:00028090  _EVP_PKEY_set_type
0001:000280ba* _EVP_PKEY_set_type_str
0001:000280e3  _EVP_PKEY_assign
0001:0002811b* _EVP_PKEY_get0
0001:00028126  _EVP_PKEY_set1_RSA
0001:0002815f  _EVP_PKEY_get1_RSA
0001:000281b8  _EVP_PKEY_set1_DSA
0001:000281f1  _EVP_PKEY_get1_DSA
0001:0002824a  _EVP_PKEY_set1_EC_KEY
0001:00028283  _EVP_PKEY_get1_EC_KEY
0001:000282de* _EVP_PKEY_set1_DH
0001:00028317* _EVP_PKEY_get1_DH
0001:00028370  _EVP_PKEY_type
0001:000283b9  _EVP_PKEY_id
0001:000283c3* _EVP_PKEY_base_id
0001:000283d8  _EVP_PKEY_free
0001:00028534  _EVP_PKEY_print_public
0001:000285a8  _EVP_PKEY_print_private
0001:0002861b  _EVP_PKEY_print_params
0001:00028683  _EVP_PKEY_get_default_digest_nid
Module: U:\extras\lib\libcrypto.lib(p5_crpt.obj)
0001:000286e0* _PKCS5_PBE_add
0001:0002874b  _PKCS5_PBE_keyivgen
Module: U:\extras\lib\libcrypto.lib(p12_crpt.obj)
0001:00028ac0* _PKCS12_PBE_add
0001:00028ad0  _PKCS12_PBE_keyivgen
Module: U:\extras\lib\libcrypto.lib(p5_crpt2.obj)
0001:00028d60* _PKCS5_PBKDF2_HMAC
0001:00028f4d* _PKCS5_PBKDF2_HMAC_SHA1
0001:00028fb3  _PKCS5_v2_PBE_keyivgen
Module: U:\extras\lib\libcrypto.lib(md4_dgst.obj)
0001:000294f0  _MD4_Update
0001:00029896* _md4_block_data_order
0001:000296a7* _MD4_Transform
0001:000296c9  _MD4_Final
0001:00029820* _MD4_version
0001:00029847  _MD4_Init
Module: U:\extras\lib\libcrypto.lib(rsa_sign.obj)
0001:0002a1bb  _RSA_sign
0001:0002a4cd  _int_rsa_verify
0001:0002a949  _RSA_verify
Module: U:\extras\lib\libcrypto.lib(md5_dgst.obj)
0001:0002a9e0  _MD5_Update
0001:0002ad86* _md5_block_data_order
0001:0002ab97* _MD5_Transform
0001:0002abb9  _MD5_Final
0001:0002ad10* _MD5_version
0001:0002ad37  _MD5_Init
Module: U:\extras\lib\libcrypto.lib(sha_dgst.obj)
0001:0002ba20* _SHA_version
0001:0002ba47  _SHA_Update
0001:0002bbfe* _SHA_Transform
0001:0002bc20  _SHA_Final
0001:0002bdee  _SHA_Init
Module: U:\extras\lib\libcrypto.lib(sha1dgst.obj)
0001:0002e260* _SHA1_version
0001:0002e288  _SHA1_Update
0001:0002e43f* _SHA1_Transform
0001:0002e461  _SHA1_Final
0001:0002e62f  _SHA1_Init
Module: U:\extras\lib\libcrypto.lib(dsa_sign.obj)
0001:00030df0* _DSA_do_sign
0001:00030e17  _DSA_sign
0001:00030e8c  _DSA_sign_setup
Module: U:\extras\lib\libcrypto.lib(dsa_vrf.obj)
0001:00030ec0* _DSA_do_verify
0001:00030eee  _DSA_verify
Module: U:\extras\lib\libcrypto.lib(sha256.obj)
0001:00030f70* _SHA256_version
0001:00030f9b  _SHA224_Init
0001:0003101c  _SHA256_Init
0001:0003109d* _SHA224
0001:000311a0  _SHA256_Update
0001:00031379  _SHA256_Final
0001:00031101* _SHA256
0001:00031165* _SHA224_Update
0001:00031186* _SHA224_Final
0001:00031357* _SHA256_Transform
Module: U:\extras\lib\libcrypto.lib(sha512.obj)
0001:000339a0* _SHA512_version
0001:000339cb  _SHA384_Init
0001:00033a98  _SHA512_Init
0001:00033b65  _SHA512_Final
0001:00033f77* _SHA384_Final
0001:00033f91  _SHA512_Update
0001:0003414a* _SHA384_Update
0001:0003416b* _SHA512_Transform
0001:0003418d* _SHA384
0001:000341fd* _SHA512
Module: U:\extras\lib\libcrypto.lib(ecs_sign.obj)
0001:00034e60* _ECDSA_do_sign
0001:00034e91* _ECDSA_do_sign_ex
0001:00034ee1  _ECDSA_sign
0001:00034f27* _ECDSA_sign_ex
0001:00034faa  _ECDSA_sign_setup
Module: U:\extras\lib\libcrypto.lib(ecs_vrf.obj)
0001:00035000* _ECDSA_do_verify
0001:00035049  _ECDSA_verify
Module: U:\extras\lib\libcrypto.lib(mdc2dgst.obj)
0001:000350c0  _MDC2_Init
0001:0003511c  _MDC2_Update
0001:000354c9  _MDC2_Final
Module: U:\extras\lib\libcrypto.lib(rsa_saos.obj)
0001:0003559b  _RSA_sign_ASN1_OCTET_STRING
0001:000356f5  _RSA_verify_ASN1_OCTET_STRING
Module: U:\extras\lib\libcrypto.lib(rmd_dgst.obj)
0001:000358a0  _RIPEMD160_Update
0001:00035c77* _ripemd160_block_data_order
0001:00035a57* _RIPEMD160_Transform
0001:00035a79  _RIPEMD160_Final
0001:00035bf0* _RMD160_version
0001:00035c1e  _RIPEMD160_Init
Module: U:\extras\lib\libcrypto.lib(wp_dgst.obj)
0001:000389d0  _WHIRLPOOL_Init
0001:000389f8  _WHIRLPOOL_Update
0001:00038a66* _WHIRLPOOL_BitUpdate
0001:00038e9f  _WHIRLPOOL_Final
0001:0003903f* _WHIRLPOOL
Module: U:\extras\lib\libcrypto.lib(tasn_fre.obj)
0001:000390a0  _ASN1_item_free
0001:000390c2  _ASN1_item_ex_free
0001:00039473  _ASN1_template_free
0001:00039519  _ASN1_primitive_free
Module: U:\extras\lib\libcrypto.lib(tasn_dec.obj)
0001:000396e0  _ASN1_tag2bit
0001:00039702  _ASN1_item_d2i
0001:000397cb  _ASN1_item_ex_d2i
0001:00039770* _ASN1_template_d2i
0001:0003aff4* _asn1_ex_c2i
Module: U:\extras\lib\libcrypto.lib(tasn_enc.obj)
0001:0003bb50  _ASN1_item_ndef_i2d
0001:0003bb79  _ASN1_item_i2d
0001:0003bc94  _ASN1_item_ex_i2d
0001:0003c1bc* _ASN1_template_i2d
0001:0003c9a1* _asn1_ex_i2c
Module: U:\extras\lib\libcrypto.lib(tasn_new.obj)
0001:0003cc40  _ASN1_item_new
0001:0003cc6f  _ASN1_item_ex_new
0001:0003d1bc* _ASN1_template_new
0001:0003d2d2* _ASN1_primitive_new
Module: U:\extras\lib\libcrypto.lib(bn_asm.obj)
0001:0003d4c0  _bn_mul_add_words
0001:0003d990  _bn_mul_words
0001:0003ddad  _bn_sqr_words
0001:0003e004  _bn_div_words
0001:0003e191  _bn_add_words
0001:0003e343  _bn_sub_words
0001:0003e4ea  _bn_mul_comba8
0001:00043d2c  _bn_mul_comba4
0001:000451be  _bn_sqr_comba8
0001:0004875c  _bn_sqr_comba4
Module: U:\extras\lib\libcrypto.lib(bss_file.obj)
0001:00049387  _BIO_new_file
0001:0004953f  _BIO_s_file
0001:000494e3  _BIO_new_fp
Module: U:\extras\lib\libcrypto.lib(ex_data.obj)
0001:00049c1d* _CRYPTO_get_ex_data_implementation
0001:00049c38* _CRYPTO_set_ex_data_implementation
0001:0004a9c1  _CRYPTO_get_ex_data
0001:0004a8dc  _CRYPTO_set_ex_data
0001:0004a7ab* _CRYPTO_ex_data_new_class
0001:0004a7ca* _CRYPTO_cleanup_all_ex_data
0001:0004a7ea  _CRYPTO_get_ex_new_index
0001:0004a840  _CRYPTO_new_ex_data
0001:0004a874  _CRYPTO_dup_ex_data
0001:0004a8a8  _CRYPTO_free_ex_data
Module: U:\extras\lib\libcrypto.lib(tb_asnmth.obj)
0001:0004aa10* _ENGINE_unregister_pkey_asn1_meths
0001:0004aa3f* _ENGINE_register_pkey_asn1_meths
0001:0004aab7* _ENGINE_register_all_pkey_asn1_meths
0001:0004aae8* _ENGINE_set_default_pkey_asn1_meths
0001:0004ab60  _ENGINE_get_pkey_asn1_meth_engine
0001:0004ab87  _ENGINE_get_pkey_asn1_meth
0001:0004abfe* _ENGINE_get_pkey_asn1_meths
0001:0004ac09* _ENGINE_set_pkey_asn1_meths
0001:0004ac1c  _engine_pkey_asn1_meths_free
0001:0004aca7* _ENGINE_get_pkey_asn1_meth_str
0001:0004ae4e  _ENGINE_pkey_asn1_find_str
Module: U:\extras\lib\libcrypto.lib(rand_lib.obj)
0001:0004aef0  _RAND_set_rand_method
0001:0004af25* _RAND_get_rand_method
0001:0004af8e* _RAND_set_rand_engine
0001:0004aff7* _RAND_cleanup
0001:0004b02b  _RAND_seed
0001:0004b05e  _RAND_add
0001:0004b0ad  _RAND_bytes
0001:0004b0e9  _RAND_pseudo_bytes
0001:0004b125  _RAND_status
Module: U:\extras\lib\libcrypto.lib(eng_ctrl.obj)
0001:0004b592* _ENGINE_ctrl
0001:0004b77b* _ENGINE_cmd_is_executable
0001:0004b813* _ENGINE_ctrl_cmd
0001:0004b916  _ENGINE_ctrl_cmd_string
Module: U:\extras\lib\libcrypto.lib(rsa_x931.obj)
0001:0004bc9b  _RSA_padding_add_X931
0001:0004bd69  _RSA_padding_check_X931
0001:0004bef3  _RSA_X931_hash_id
Module: U:\extras\lib\libcrypto.lib(rsa_lib.obj)
0001:0004bf50* _RSA_version
0001:0004bf77  _RSA_new
0001:0004c044* _RSA_new_method
0001:0004bf91* _RSA_set_default_method
0001:0004bf9e* _RSA_get_default_method
0001:0004bfbe* _RSA_get_method
0001:0004bfc9* _RSA_set_method
0001:0004c304  _RSA_free
0001:0004c4bd  _RSA_up_ref
0001:0004c500* _RSA_get_ex_new_index
0001:0004c537* _RSA_set_ex_data
0001:0004c55b* _RSA_get_ex_data
0001:0004c578  _RSA_size
0001:0004c59b  _RSA_public_encrypt
0001:0004c5d0  _RSA_private_encrypt
0001:0004c605  _RSA_private_decrypt
0001:0004c63a  _RSA_public_decrypt
0001:0004c66f* _RSA_flags
0001:0004c68a* _RSA_blinding_off
0001:0004c6d6* _RSA_blinding_on
0001:0004c855  _RSA_setup_blinding
0001:0004cada* _RSA_memory_lock
Module: U:\extras\lib\libcrypto.lib(rsa_pss.obj)
0001:0004cce2  _RSA_verify_PKCS1_PSS
0001:0004d133  _RSA_padding_add_PKCS1_PSS
Module: U:\extras\lib\libcrypto.lib(pmeth_gn.obj)
0001:0004d46b* _EVP_PKEY_paramgen_init
0001:0004d504* _EVP_PKEY_paramgen
0001:0004d5f6* _EVP_PKEY_keygen_init
0001:0004d68f* _EVP_PKEY_keygen
0001:0004d781* _EVP_PKEY_CTX_set_cb
0001:0004d78f* _EVP_PKEY_CTX_get_cb
0001:0004d7d2  _evp_pkey_set_cb_translate
0001:0004d7fc* _EVP_PKEY_CTX_get_keygen_info
0001:0004d837* _EVP_PKEY_new_mac_key
Module: U:\extras\lib\libcrypto.lib(rsa_gen.obj)
0001:0004d8e0  _RSA_generate_key_ex
Module: U:\extras\lib\libcrypto.lib(dh_lib.obj)
0001:0004e160* _DH_version
0001:0004e192* _DH_set_default_method
0001:0004e19f* _DH_get_default_method
0001:0004e1bf* _DH_set_method
0001:0004e230  _DH_new
0001:0004e24d* _DH_new_method
0001:0004e4c1  _DH_free
0001:0004e632  _DH_up_ref
0001:0004e675* _DH_get_ex_new_index
0001:0004e6ac* _DH_set_ex_data
0001:0004e6d0* _DH_get_ex_data
0001:0004e6ed  _DH_size
Module: U:\extras\lib\libcrypto.lib(dh_gen.obj)
0001:0004e710  _DH_generate_parameters_ex
Module: U:\extras\lib\libcrypto.lib(dh_key.obj)
0001:0004ea10  _DH_generate_key
0001:0004ea29  _DH_compute_key
0001:0004ea62  _DH_OpenSSL
Module: U:\extras\lib\libcrypto.lib(dsa_lib.obj)
0001:0004f000* _DSA_version
0001:0004f027* _DSA_set_default_method
0001:0004f034* _DSA_get_default_method
0001:0004f054  _DSA_new
0001:0004f0e3* _DSA_new_method
0001:0004f068* _DSA_set_method
0001:0004f343  _DSA_free
0001:0004f49c  _DSA_up_ref
0001:0004f4df  _DSA_size
0001:0004f55b* _DSA_get_ex_new_index
0001:0004f592* _DSA_set_ex_data
0001:0004f5b6* _DSA_get_ex_data
0001:0004f5d3* _DSA_dup_DH
Module: U:\extras\lib\libcrypto.lib(dsa_gen.obj)
0001:0004f6f0* _DSA_generate_parameters_ex
0001:0004f7c9  _dsa_builtin_paramgen
Module: U:\extras\lib\libcrypto.lib(dsa_key.obj)
0001:00050100  _DSA_generate_key
Module: U:\extras\lib\libcrypto.lib(ec_lib.obj)
0001:0005031f  _EC_GROUP_new
0001:0005048f  _EC_GROUP_free
0001:00051427  _EC_EX_DATA_free_all_data
0001:000515e0  _EC_POINT_free
0001:00050525  _EC_GROUP_clear_free
0001:0005147b* _EC_EX_DATA_clear_free_all_data
0001:00051618  _EC_POINT_clear_free
0001:00050604  _EC_GROUP_copy
0001:000511d2  _EC_EX_DATA_set_data
0001:000514cf  _EC_POINT_new
0001:00051681  _EC_POINT_copy
0001:00050901  _EC_GROUP_dup
0001:00050982  _EC_GROUP_method_of
0001:0005098c  _EC_METHOD_get_field_type
0001:00050996  _EC_GROUP_set_generator
0001:00050aa6  _EC_GROUP_get0_generator
0001:00050ab1  _EC_GROUP_get_order
0001:00050ae7  _EC_GROUP_get_cofactor
0001:00050b1d  _EC_GROUP_set_curve_name
0001:00050b2b  _EC_GROUP_get_curve_name
0001:00050b36  _EC_GROUP_set_asn1_flag
0001:00050b44  _EC_GROUP_get_asn1_flag
0001:00050b4f  _EC_GROUP_set_point_conversion_form
0001:00050b5d  _EC_GROUP_get_point_conversion_form
0001:00050b68  _EC_GROUP_set_seed
0001:00050c0b  _EC_GROUP_get0_seed
0001:00050c16  _EC_GROUP_get_seed_len
0001:00050c21  _EC_GROUP_set_curve_GFp
0001:00050c94  _EC_GROUP_get_curve_GFp
0001:00050d07  _EC_GROUP_set_curve_GF2m
0001:00050d7a  _EC_GROUP_get_curve_GF2m
0001:00050ded  _EC_GROUP_get_degree
0001:00050e44* _EC_GROUP_check_discriminant
0001:00050ea2  _EC_GROUP_cmp
0001:000522ce  _EC_POINT_cmp
0001:000512cd  _EC_EX_DATA_get_data
0001:00051319  _EC_EX_DATA_free_data
0001:000513a0* _EC_EX_DATA_clear_free_data
0001:0005172f  _EC_POINT_dup
0001:0005178f* _EC_POINT_method_of
0001:00051799  _EC_POINT_set_to_infinity
0001:00051838  _EC_POINT_set_Jprojective_coordinates_GFp
0001:000518f3* _EC_POINT_get_Jprojective_coordinates_GFp
0001:000519ae  _EC_POINT_set_affine_coordinates_GFp
0001:00051a62  _EC_POINT_set_affine_coordinates_GF2m
0001:00051b16  _EC_POINT_get_affine_coordinates_GFp
0001:00051bca  _EC_POINT_get_affine_coordinates_GF2m
0001:00051c7e  _EC_POINT_set_compressed_coordinates_GFp
0001:00051d32  _EC_POINT_set_compressed_coordinates_GF2m
0001:00051de6  _EC_POINT_point2oct
0001:00051ea1  _EC_POINT_oct2point
0001:00051f55  _EC_POINT_add
0001:00052028  _EC_POINT_dbl
0001:000520e3  _EC_POINT_invert
0001:00052189  _EC_POINT_is_at_infinity
0001:00052228  _EC_POINT_is_on_curve
0001:00052389  _EC_POINT_make_affine
0001:0005242f  _EC_POINTs_make_affine
0001:000524fb* _EC_POINTs_mul
0001:00052580  _EC_POINT_mul
0001:000525de  _EC_GROUP_precompute_mult
0001:00052630  _EC_GROUP_have_precompute_mult
Module: U:\extras\lib\libcrypto.lib(ecs_lib.obj)
0001:00052680* _ECDSA_version
0001:000526a9* _ECDSA_set_default_method
0001:000526b6* _ECDSA_get_default_method
0001:000526d6* _ECDSA_set_method
0001:00052900  _ecdsa_check
0001:0005297e  _ECDSA_size
0001:00052a7f* _ECDSA_get_ex_new_index
0001:00052ab6* _ECDSA_set_ex_data
0001:00052af5* _ECDSA_get_ex_data
Module: U:\extras\lib\libcrypto.lib(ec_key.obj)
0001:00052b39  _EC_KEY_new
0001:00052beb* _EC_KEY_new_by_curve_name
0001:00052c38  _EC_KEY_free
0001:00052cfb* _EC_KEY_copy
0001:00052f46* _EC_KEY_dup
0001:00052f8e  _EC_KEY_up_ref
0001:00052fd1  _EC_KEY_generate_key
0001:000531ba* _EC_KEY_check_key
0001:00053541  _EC_KEY_get0_group
0001:0005354c  _EC_KEY_set_group
0001:0005358b  _EC_KEY_get0_private_key
0001:00053596* _EC_KEY_set_private_key
0001:000535d5  _EC_KEY_get0_public_key
0001:000535e0  _EC_KEY_set_public_key
0001:00053629  _EC_KEY_get_enc_flags
0001:00053634  _EC_KEY_set_enc_flags
0001:00053642  _EC_KEY_get_conv_form
0001:0005364d* _EC_KEY_set_conv_form
0001:0005367d  _EC_KEY_get_key_method_data
0001:000536a8  _EC_KEY_insert_key_method_data
0001:0005374e* _EC_KEY_set_asn1_flag
0001:00053775* _EC_KEY_precompute_mult
Module: U:\extras\lib\libcrypto.lib(ech_key.obj)
0001:000537b0  _ECDH_compute_key
Module: U:\extras\lib\libcrypto.lib(ec_curve.obj)
0001:00057933  _EC_GROUP_new_by_curve_name
0001:000579e8* _EC_get_builtin_curves
Module: U:\extras\lib\libcrypto.lib(hmac.obj)
0001:00057ab9  _HMAC_Init_ex
0001:00057d6b* _HMAC_Init
0001:00057e70  _HMAC_CTX_init
0001:00057db2  _HMAC_Update
0001:00057dd6  _HMAC_Final
0001:00057ea2  _HMAC_CTX_copy
0001:00057f47  _HMAC_CTX_cleanup
0001:00057f94  _HMAC
0001:00058040  _HMAC_CTX_set_flags
Module: U:\extras\lib\libcrypto.lib(a_octet.obj)
0001:00058090  _ASN1_OCTET_STRING_dup
0001:000580a3  _ASN1_OCTET_STRING_cmp
0001:000580bd  _ASN1_OCTET_STRING_set
Module: U:\extras\lib\libcrypto.lib(v3_utl.obj)
0001:00058171  _X509V3_add_value
0001:000582b8  _X509V3_add_value_uchar
0001:000582d9  _X509V3_conf_free
0001:00058346  _X509V3_add_value_bool
0001:0005838a* _X509V3_add_value_bool_nf
0001:000583b9  _i2s_ASN1_ENUMERATED
0001:00058446  _i2s_ASN1_INTEGER
0001:000584d3  _s2i_ASN1_INTEGER
0001:00058683  _X509V3_add_value_int
0001:0005871e  _X509V3_get_value_bool
0001:000588e3  _X509V3_get_value_int
0001:0005895f  _X509V3_parse_list
0001:00058cce  _hex_to_string
0001:00058db2  _string_to_hex
0001:00059006  _name_cmp
0001:00059084* _X509_get1_email
0001:000590e6* _X509_get1_ocsp
0001:000591a7* _X509_REQ_get1_email
0001:000593f3* _X509_email_free
0001:0005940f  _a2i_IPADDRESS
0001:000595ae* _a2i_ipadd
0001:00059480  _a2i_IPADDRESS_NC
0001:00059a44  _X509V3_NAME_from_section
Module: U:\extras\lib\libcrypto.lib(ameth_lib.obj)
0001:00059be0* _EVP_PKEY_asn1_get_count
0001:00059c0b* _EVP_PKEY_asn1_get0
0001:00059ce1  _EVP_PKEY_asn1_find
0001:00059d57  _EVP_PKEY_asn1_find_str
0001:00059e41* _EVP_PKEY_asn1_add0
0001:00059ea5* _EVP_PKEY_asn1_add_alias
0001:00059f78* _EVP_PKEY_asn1_new
0001:00059ef4* _EVP_PKEY_asn1_get0_info
0001:00059f61* _EVP_PKEY_get0_asn1
0001:0005a1ea  _EVP_PKEY_asn1_free
0001:0005a101* _EVP_PKEY_asn1_copy
0001:0005a240* _EVP_PKEY_asn1_set_public
0001:0005a27b* _EVP_PKEY_asn1_set_private
0001:0005a29b* _EVP_PKEY_asn1_set_param
0001:0005a2d6* _EVP_PKEY_asn1_set_free
0001:0005a2e4* _EVP_PKEY_asn1_set_ctrl
Module: U:\extras\lib\libcrypto.lib(x_attrib.obj)
0001:0005a360* _X509_ATTRIBUTE_SET_it
0001:0005a3c0  _X509_ATTRIBUTE_it
0001:0005a3dc* _d2i_X509_ATTRIBUTE
0001:0005a405* _i2d_X509_ATTRIBUTE
0001:0005a427  _X509_ATTRIBUTE_new
0001:0005a43b  _X509_ATTRIBUTE_free
0001:0005a456  _X509_ATTRIBUTE_dup
0001:0005a471  _X509_ATTRIBUTE_create
Module: U:\extras\lib\libcrypto.lib(p5_pbe.obj)
0001:0005a5a0* _PBEPARAM_it
0001:0005a5bc  _d2i_PBEPARAM
0001:0005a5e5* _i2d_PBEPARAM
0001:0005a607* _PBEPARAM_new
0001:0005a61b  _PBEPARAM_free
0001:0005a63f* _PKCS5_pbe_set0_algor
0001:0005a854  _PKCS5_pbe_set
Module: U:\extras\lib\libcrypto.lib(evp_enc.obj)
0001:0005a8e0* _EVP_version
0001:0005a907  _EVP_CIPHER_CTX_init
0001:0005a934* _EVP_CIPHER_CTX_new
0001:0005a96f* _EVP_CipherInit
0001:0005aa4e  _EVP_CipherInit_ex
0001:0005b79e  _EVP_CIPHER_CTX_cleanup
0001:0005b925  _EVP_CIPHER_CTX_ctrl
0001:0005ae7a  _EVP_CipherUpdate
0001:0005b052  _EVP_EncryptUpdate
0001:0005b3f4  _EVP_DecryptUpdate
0001:0005aedc  _EVP_CipherFinal_ex
0001:0005b2c1  _EVP_EncryptFinal_ex
0001:0005b587  _EVP_DecryptFinal_ex
0001:0005af22* _EVP_CipherFinal
0001:0005b285* _EVP_EncryptFinal
0001:0005b560* _EVP_DecryptFinal
0001:0005af68* _EVP_EncryptInit
0001:0005af98  _EVP_EncryptInit_ex
0001:0005afcf* _EVP_DecryptInit
0001:0005afff  _EVP_DecryptInit_ex
0001:0005b77a* _EVP_CIPHER_CTX_free
0001:0005b84c  _EVP_CIPHER_CTX_set_key_length
0001:0005b8f1* _EVP_CIPHER_CTX_set_padding
0001:0005ba0f  _EVP_CIPHER_CTX_rand_key
0001:0005ba71  _EVP_CIPHER_CTX_copy
Module: U:\extras\lib\libcrypto.lib(p12_key.obj)
0001:0005bc2a  _PKCS12_key_gen_asc
0001:0005bd1b* _PKCS12_key_gen_uni
Module: U:\extras\lib\libcrypto.lib(p5_pbev2.obj)
0001:0005c280* _PBE2PARAM_it
0001:0005c29c  _d2i_PBE2PARAM
0001:0005c2c5* _i2d_PBE2PARAM
0001:0005c2e7* _PBE2PARAM_new
0001:0005c2fb  _PBE2PARAM_free
0001:0005c390* _PBKDF2PARAM_it
0001:0005c3ac  _d2i_PBKDF2PARAM
0001:0005c3d5* _i2d_PBKDF2PARAM
0001:0005c3f7* _PBKDF2PARAM_new
0001:0005c40b  _PBKDF2PARAM_free
0001:0005c431* _PKCS5_pbe2_set_iv
0001:0005c96d  _PKCS5_pbe2_set
Module: U:\extras\lib\libcrypto.lib(x_sig.obj)
0001:0005ca00  _X509_SIG_it
0001:0005ca1c  _d2i_X509_SIG
0001:0005ca45  _i2d_X509_SIG
0001:0005ca67  _X509_SIG_new
0001:0005ca7b  _X509_SIG_free
Module: U:\extras\lib\libcrypto.lib(dsa_asn1.obj)
0001:0005cb90* _DSA_SIG_it
0001:0005cbac  _d2i_DSA_SIG
0001:0005cbd5  _i2d_DSA_SIG
0001:0005cbf7  _DSA_SIG_new
0001:0005cc0b  _DSA_SIG_free
0001:0005cd40* _DSAPrivateKey_it
0001:0005cd5c  _d2i_DSAPrivateKey
0001:0005cd85  _i2d_DSAPrivateKey
0001:0005ce10* _DSAparams_it
0001:0005ce2c  _d2i_DSAparams
0001:0005ce55  _i2d_DSAparams
0001:0005ced0* _dsa_pub_internal_it
0001:0005cf40* _DSAPublicKey_it
0001:0005cf5c* _d2i_DSAPublicKey
0001:0005cf85  _i2d_DSAPublicKey
0001:0005cfa7* _DSAparams_dup
Module: U:\extras\lib\libcrypto.lib(ecs_asn1.obj)
0001:0005d020* _ECDSA_SIG_it
0001:0005d03c  _d2i_ECDSA_SIG
0001:0005d065  _i2d_ECDSA_SIG
0001:0005d087  _ECDSA_SIG_new
0001:0005d09b  _ECDSA_SIG_free
Module: U:\extras\lib\libcrypto.lib(set_key.obj)
0001:0005d1c0  _DES_set_odd_parity
0001:0005d1f5* _DES_check_key_parity
0001:0005d2c0* _DES_is_weak_key
0001:0005db10* _DES_set_key
0001:0005db4c* _DES_set_key_checked
0001:0005db97  _DES_set_key_unchecked
0001:0005de84* _DES_key_sched
0002:000033e0* __shadow_DES_check_key
Module: U:\extras\lib\libcrypto.lib(des_enc.obj)
0001:0005dee0* _DES_SPtrans
0001:0005e6e0  _DES_encrypt1
0001:00061409* _DES_encrypt2
0001:0006404a* _DES_encrypt3
0001:000641c1* _DES_decrypt3
0001:00064338* _DES_ncbc_encrypt
0001:00064a98* _DES_ede3_cbc_encrypt
Module: U:\extras\lib\libcrypto.lib(wp_block.obj)
0001:00066240  _whirlpool_block
Module: U:\extras\lib\libcrypto.lib(tasn_utl.obj)
0001:000683c0  _asn1_get_choice_selector
0001:000683e0  _asn1_set_choice_selector
0001:00068419  _asn1_do_lock
0001:00068509  _asn1_enc_init
0001:00068549  _asn1_enc_free
0001:0006859f  _asn1_enc_save
0001:00068644  _asn1_enc_restore
0001:000686c8  _asn1_get_field_ptr
0001:000686f9  _asn1_do_adb
Module: U:\extras\lib\libcrypto.lib(a_bitstr.obj)
0001:00068810  _ASN1_BIT_STRING_set
0001:00068831  _i2c_ASN1_BIT_STRING
0001:000689f1  _c2i_ASN1_BIT_STRING
0001:00068bbd  _ASN1_BIT_STRING_set_bit
0001:00068d9f  _ASN1_BIT_STRING_get_bit
0001:00068e14* _ASN1_BIT_STRING_check
Module: U:\extras\lib\libcrypto.lib(tb_rand.obj)
0001:00068e94* _ENGINE_unregister_RAND
0001:00068ec3* _ENGINE_register_RAND
0001:00068f0f* _ENGINE_register_all_RAND
0001:00068f40* _ENGINE_set_default_RAND
0001:00068f8c  _ENGINE_get_default_RAND
0001:00068fa9  _ENGINE_get_RAND
0001:00068fb4* _ENGINE_set_RAND
Module: U:\extras\lib\libcrypto.lib(md_rand.obj)
0001:00068fd0* _RAND_version
0001:00068ff8  _RAND_SSLeay
0002:00000aa0* _rand_ssleay_meth
Module: U:\extras\lib\libcrypto.lib(rsa_eay.obj)
0001:00069c48  _RSA_PKCS1_SSLeay
Module: U:\extras\lib\libcrypto.lib(tb_rsa.obj)
0001:0006bd04* _ENGINE_unregister_RSA
0001:0006bd33* _ENGINE_register_RSA
0001:0006bd7f* _ENGINE_register_all_RSA
0001:0006bdb0* _ENGINE_set_default_RSA
0001:0006bdfc  _ENGINE_get_default_RSA
0001:0006be19  _ENGINE_get_RSA
0001:0006be24* _ENGINE_set_RSA
Module: U:\extras\lib\libcrypto.lib(bn_blind.obj)
0001:0006be4b* _BN_BLINDING_new
0001:0006bf87  _BN_BLINDING_free
0001:0006c001* _BN_BLINDING_update
0001:0006c3a4  _BN_BLINDING_create_param
0001:0006c17c* _BN_BLINDING_convert
0001:0006c1a5  _BN_BLINDING_convert_ex
0001:0006c291* _BN_BLINDING_invert
0001:0006c2ba  _BN_BLINDING_invert_ex
0001:0006c367* _BN_BLINDING_get_thread_id
0001:0006c372* _BN_BLINDING_set_thread_id
0001:0006c380  _BN_BLINDING_thread_id
0001:0006c38b* _BN_BLINDING_get_flags
0001:0006c396* _BN_BLINDING_set_flags
Module: U:\extras\lib\libcrypto.lib(bn_ctx.obj)
0001:0006c610* _BN_CTX_init
0001:0006c658  _BN_CTX_new
0001:0006c6f2  _BN_CTX_free
0001:0006c727  _BN_CTX_start
0001:0006c7ab  _BN_CTX_end
0001:0006c817  _BN_CTX_get
Module: U:\extras\lib\libcrypto.lib(bn_add.obj)
0001:0006ccf0  _BN_add
0001:0006cf59  _BN_usub
0001:0006cdcb  _BN_uadd
0001:0006d172  _BN_sub
Module: U:\extras\lib\libcrypto.lib(bn_mul.obj)
0001:0006d2e0* _bn_sub_part_words
0001:0006d624* _bn_add_part_words
0001:0006da6c* _bn_mul_recursive
0001:0006f72c* _bn_mul_normal
0001:0006e19a* _bn_mul_part_recursive
0001:0006e9ba* _bn_mul_low_recursive
0001:0006f8cf* _bn_mul_low_normal
0001:0006eb9b* _bn_mul_high
0001:0006f2ce  _BN_mul
Module: U:\extras\lib\libcrypto.lib(bn_gcd.obj)
0001:0006f9e0  _BN_gcd
0001:0006fcd0  _BN_mod_inverse
Module: U:\extras\lib\libcrypto.lib(rsa_oaep.obj)
0001:0007094b  _RSA_padding_add_PKCS1_OAEP
0001:00070bd5  _RSA_padding_check_PKCS1_OAEP
0001:00070ee6  _PKCS1_MGF1
Module: U:\extras\lib\libcrypto.lib(bn_prime.obj)
0001:000720a0  _BN_GENCB_call
0001:00072120  _BN_generate_prime_ex
0001:0007246b  _BN_is_prime_fasttest_ex
0001:0007243b  _BN_is_prime_ex
Module: U:\extras\lib\libcrypto.lib(bn_div.obj)
0001:00072f19  _BN_div
Module: U:\extras\lib\libcrypto.lib(tb_dh.obj)
0001:00073c64* _ENGINE_unregister_DH
0001:00073c93* _ENGINE_register_DH
0001:00073cdf* _ENGINE_register_all_DH
0001:00073d10* _ENGINE_set_default_DH
0001:00073d5c  _ENGINE_get_default_DH
0001:00073d79  _ENGINE_get_DH
0001:00073d84* _ENGINE_set_DH
Module: U:\extras\lib\libcrypto.lib(bn_mont.obj)
0001:00073da0  _BN_mod_mul_montgomery
0001:00074330  _BN_from_montgomery
0001:000743a8  _BN_MONT_CTX_new
0001:000743f4* _BN_MONT_CTX_init
0001:0007444f  _BN_MONT_CTX_free
0001:000744a2  _BN_MONT_CTX_set
0001:00074713  _BN_MONT_CTX_copy
0001:000747b9  _BN_MONT_CTX_set_locked
Module: U:\extras\lib\libcrypto.lib(bn_rand.obj)
0001:00074b92  _BN_rand
0001:00074bc2  _BN_pseudo_rand
0001:00074bf2* _BN_bntest_rand
0001:00074e80  _BN_rand_range
0001:00074ea2  _BN_pseudo_rand_range
Module: U:\extras\lib\libcrypto.lib(dh_check.obj)
0001:00074ed0* _DH_check
0001:000750ad  _DH_check_pub_key
Module: U:\extras\lib\libcrypto.lib(bn_exp.obj)
0001:00075199* _BN_exp
0001:00075359  _BN_mod_exp
0001:000765b6  _BN_mod_exp_mont_word
0001:000758fd  _BN_mod_exp_mont
0001:00075443* _BN_mod_exp_recp
0001:0007603c* _BN_mod_exp_mont_consttime
0001:00076adc* _BN_mod_exp_simple
Module: U:\extras\lib\libcrypto.lib(dsa_ossl.obj)
0001:00076f03  _DSA_OpenSSL
Module: U:\extras\lib\libcrypto.lib(tb_dsa.obj)
0001:00077a34* _ENGINE_unregister_DSA
0001:00077a63* _ENGINE_register_DSA
0001:00077aaf* _ENGINE_register_all_DSA
0001:00077ae0* _ENGINE_set_default_DSA
0001:00077b2c  _ENGINE_get_default_DSA
0001:00077b49  _ENGINE_get_DSA
0001:00077b54* _ENGINE_set_DSA
Module: U:\extras\lib\libcrypto.lib(ec_mult.obj)
0001:00078182  _ec_wNAF_mul
0001:00078f5b  _ec_wNAF_precompute_mult
0001:00079592  _ec_wNAF_have_precompute_mult
Module: U:\extras\lib\libcrypto.lib(ecs_ossl.obj)
0001:000795e5  _ECDSA_OpenSSL
Module: U:\extras\lib\libcrypto.lib(tb_ecdsa.obj)
0001:0007a684* _ENGINE_unregister_ECDSA
0001:0007a6b3* _ENGINE_register_ECDSA
0001:0007a6ff* _ENGINE_register_all_ECDSA
0001:0007a730* _ENGINE_set_default_ECDSA
0001:0007a77c  _ENGINE_get_default_ECDSA
0001:0007a799  _ENGINE_get_ECDSA
0001:0007a7a4* _ENGINE_set_ECDSA
Module: U:\extras\lib\libcrypto.lib(ech_lib.obj)
0001:0007a7c0* _ECDH_version
0001:0007a7e8* _ECDH_set_default_method
0001:0007a7f5* _ECDH_get_default_method
0001:0007a815* _ECDH_set_method
0001:0007aa3f  _ecdh_check
0001:0007aabd* _ECDH_get_ex_new_index
0001:0007aaf4* _ECDH_set_ex_data
0001:0007ab33* _ECDH_get_ex_data
Module: U:\extras\lib\libcrypto.lib(ec_cvt.obj)
0001:0007ab70  _EC_GROUP_new_curve_GFp
0001:0007ac83  _EC_GROUP_new_curve_GF2m
Module: U:\extras\lib\libcrypto.lib(a_enum.obj)
0001:0007acf9* _ASN1_ENUMERATED_set
0001:0007ae35  _ASN1_ENUMERATED_get
0001:0007aedf* _BN_to_ASN1_ENUMERATED
0001:0007b035  _ASN1_ENUMERATED_to_BN
Module: U:\extras\lib\libcrypto.lib(x509_ext.obj)
0001:0007b0c0* _X509_CRL_get_ext_count
0001:0007b0d8  _X509_CRL_get_ext_by_NID
0001:0007b0fe* _X509_CRL_get_ext_by_OBJ
0001:0007b124* _X509_CRL_get_ext_by_critical
0001:0007b14a  _X509_CRL_get_ext
0001:0007b169* _X509_CRL_delete_ext
0001:0007b188  _X509_CRL_get_ext_d2i
0001:0007b1b5* _X509_CRL_add1_ext_i2d
0001:0007b1e9* _X509_CRL_add_ext
0001:0007b217  _X509_get_ext_count
0001:0007b22f  _X509_get_ext_by_NID
0001:0007b255* _X509_get_ext_by_OBJ
0001:0007b27b* _X509_get_ext_by_critical
0001:0007b2a1  _X509_get_ext
0001:0007b2c0* _X509_delete_ext
0001:0007b2df* _X509_add_ext
0001:0007b30d  _X509_get_ext_d2i
0001:0007b33a* _X509_add1_ext_i2d
0001:0007b36e* _X509_REVOKED_get_ext_count
0001:0007b384* _X509_REVOKED_get_ext_by_NID
0001:0007b3a8* _X509_REVOKED_get_ext_by_OBJ
0001:0007b3cc* _X509_REVOKED_get_ext_by_critical
0001:0007b3f0* _X509_REVOKED_get_ext
0001:0007b40d* _X509_REVOKED_delete_ext
0001:0007b42a* _X509_REVOKED_add_ext
0001:0007b456  _X509_REVOKED_get_ext_d2i
0001:0007b481* _X509_REVOKED_add1_ext_i2d
Module: U:\extras\lib\libcrypto.lib(x509_cmp.obj)
0001:0007b4c0* _X509_issuer_and_serial_cmp
0001:0007b796  _X509_NAME_cmp
0001:0007b516* _X509_issuer_and_serial_hash
0001:0007b61d* _X509_issuer_name_cmp
0001:0007b641  _X509_subject_name_cmp
0001:0007b665  _X509_CRL_cmp
0001:0007b689  _X509_CRL_match
0001:0007b6b1  _X509_get_issuer_name
0001:0007b6be* _X509_issuer_name_hash
0001:0007b850* _X509_NAME_hash
0001:0007b6d6* _X509_issuer_name_hash_old
0001:0007b8d9* _X509_NAME_hash_old
0001:0007b6ee  _X509_get_subject_name
0001:0007b6fb  _X509_get_serialNumber
0001:0007b708* _X509_subject_name_hash
0001:0007b720* _X509_subject_name_hash_old
0001:0007b738  _X509_cmp
0001:0007b965  _X509_find_by_issuer_and_serial
0001:0007b9ed* _X509_find_by_subject
0001:0007ba4e  _X509_get_pubkey
0001:0007ba7c  _X509_get0_pubkey_bitstr
0001:0007baa4  _X509_check_private_key
Module: U:\extras\lib\libcrypto.lib(v3_genn.obj)
0001:0007bc00* _OTHERNAME_it
0001:0007bc1c* _d2i_OTHERNAME
0001:0007bc45* _i2d_OTHERNAME
0001:0007bc67  _OTHERNAME_new
0001:0007bc7b* _OTHERNAME_free
0001:0007bcf0* _EDIPARTYNAME_it
0001:0007bd0c* _d2i_EDIPARTYNAME
0001:0007bd35* _i2d_EDIPARTYNAME
0001:0007bd57* _EDIPARTYNAME_new
0001:0007bd6b* _EDIPARTYNAME_free
0001:0007bee0  _GENERAL_NAME_it
0001:0007befc* _d2i_GENERAL_NAME
0001:0007bf25* _i2d_GENERAL_NAME
0001:0007bf47  _GENERAL_NAME_new
0001:0007bf5b  _GENERAL_NAME_free
0001:0007bfc0  _GENERAL_NAMES_it
0001:0007bfdc* _d2i_GENERAL_NAMES
0001:0007c005* _i2d_GENERAL_NAMES
0001:0007c027  _GENERAL_NAMES_new
0001:0007c03b  _GENERAL_NAMES_free
0001:0007c056* _GENERAL_NAME_dup
0001:0007c07b  _GENERAL_NAME_cmp
0001:0007c19c* _OTHERNAME_cmp
0001:0007c200* _GENERAL_NAME_set0_value
0001:0007c286* _GENERAL_NAME_get0_value
0001:0007c307* _GENERAL_NAME_set0_othername
0001:0007c354* _GENERAL_NAME_get0_otherName
Module: U:\extras\lib\libcrypto.lib(v3_info.obj)
0001:0007c3a0  _v3_info
0001:0007c550* _AUTHORITY_INFO_ACCESS_it
0001:0007c3e0  _v3_sinfo
0001:0007c470  _ACCESS_DESCRIPTION_it
0001:0007c48c* _d2i_ACCESS_DESCRIPTION
0001:0007c4b5* _i2d_ACCESS_DESCRIPTION
0001:0007c4d7* _ACCESS_DESCRIPTION_new
0001:0007c4eb* _ACCESS_DESCRIPTION_free
0001:0007c56c* _d2i_AUTHORITY_INFO_ACCESS
0001:0007c595* _i2d_AUTHORITY_INFO_ACCESS
0001:0007c5b7* _AUTHORITY_INFO_ACCESS_new
0001:0007c5cb  _AUTHORITY_INFO_ACCESS_free
0001:0007ca36* _i2a_ACCESS_DESCRIPTION
Module: U:\extras\lib\libcrypto.lib(x509_req.obj)
0001:0007ca6b* _X509_to_X509_REQ
0001:0007cba1* _X509_REQ_get_pubkey
0001:0007cbcf* _X509_REQ_check_private_key
0001:0007cd44* _X509_REQ_extension_nid
0001:0007cd86* _X509_REQ_get_extension_nids
0001:0007cd90* _X509_REQ_set_extension_nids
0001:0007cd9d  _X509_REQ_get_extensions
0001:0007d035* _X509_REQ_get_attr_by_NID
0001:0007d081* _X509_REQ_get_attr
0001:0007ceb7* _X509_REQ_add_extensions_nid
0001:0007cffb  _X509_REQ_add_extensions
0001:0007d01d* _X509_REQ_get_attr_count
0001:0007d05b* _X509_REQ_get_attr_by_OBJ
0001:0007d0a0* _X509_REQ_delete_attr
0001:0007d0bf* _X509_REQ_add1_attr
0001:0007d0ee* _X509_REQ_add1_attr_by_OBJ
0001:0007d132* _X509_REQ_add1_attr_by_NID
0001:0007d176* _X509_REQ_add1_attr_by_txt
Module: U:\extras\lib\libcrypto.lib(v3_lib.obj)
0001:0007d1c9* _X509V3_EXT_add
0001:0007d2e8  _X509V3_EXT_get_nid
0001:0007d37c  _X509V3_EXT_get
0001:0007d3ac* _X509V3_EXT_add_list
0001:0007d3df* _X509V3_EXT_add_alias
0001:0007d4cb* _X509V3_EXT_cleanup
0001:0007d513* _X509V3_add_standard_extensions
0001:0007d51d  _X509V3_EXT_d2i
0001:0007d5a3  _X509V3_get_d2i
0001:0007d6cb  _X509V3_add1_i2d
Module: U:\extras\lib\libcrypto.lib(x_exten.obj)
0001:0007d930  _X509_EXTENSION_it
0001:0007d990  _X509_EXTENSIONS_it
0001:0007d9ac* _d2i_X509_EXTENSION
0001:0007d9d5* _i2d_X509_EXTENSION
0001:0007d9f7  _X509_EXTENSION_new
0001:0007da0b  _X509_EXTENSION_free
0001:0007da26* _d2i_X509_EXTENSIONS
0001:0007da4f* _i2d_X509_EXTENSIONS
0001:0007da71  _X509_EXTENSION_dup
Module: U:\extras\lib\libcrypto.lib(x509name.obj)
0001:0007da90* _X509_NAME_get_text_by_NID
0001:0007dad3* _X509_NAME_get_text_by_OBJ
0001:0007dbc7* _X509_NAME_get_index_by_OBJ
0001:0007dc46  _X509_NAME_get_entry
0001:0007e401  _X509_NAME_ENTRY_get_data
0001:0007db69  _X509_NAME_entry_count
0001:0007db8b  _X509_NAME_get_index_by_NID
0001:0007dc87  _X509_NAME_delete_entry
0001:0007dd76* _X509_NAME_add_entry_by_OBJ
0001:0007e1d2* _X509_NAME_ENTRY_create_by_OBJ
0001:0007ded4  _X509_NAME_add_entry
0001:0007dde7* _X509_NAME_add_entry_by_NID
0001:0007e14b* _X509_NAME_ENTRY_create_by_NID
0001:0007de58  _X509_NAME_add_entry_by_txt
0001:0007e0a1* _X509_NAME_ENTRY_create_by_txt
0001:0007e286* _X509_NAME_ENTRY_set_object
0001:0007e2f7* _X509_NAME_ENTRY_set_data
0001:0007e3ea  _X509_NAME_ENTRY_get_object
Module: U:\extras\lib\libcrypto.lib(conf_mod.obj)
0001:0007e485* _CONF_modules_load
0001:0007e5a6* _CONF_modules_load_file
0001:0007ef26* _CONF_get1_default_config_file
0001:0007ecd0* _CONF_modules_unload
0001:0007edaa* _CONF_modules_finish
0001:0007ee4e* _CONF_module_add
0001:0007ee87* _CONF_modules_free
0001:0007eea0* _CONF_imodule_get_name
0001:0007eeab* _CONF_imodule_get_value
0001:0007eeb6* _CONF_imodule_get_usr_data
0001:0007eec1* _CONF_imodule_set_usr_data
0001:0007eecf* _CONF_imodule_get_module
0001:0007eed9* _CONF_imodule_get_flags
0001:0007eee4* _CONF_imodule_set_flags
0001:0007eef2* _CONF_module_get_usr_data
0001:0007eefd* _CONF_module_set_usr_data
0001:0007eff7  _CONF_parse_list
Module: U:\extras\lib\libcrypto.lib(rsa_ameth.obj)
0001:0007fb60  _rsa_asn1_meths
Module: U:\extras\lib\libcrypto.lib(dh_ameth.obj)
0001:000809a7* _DHparams_print
0001:00080a00  _dh_asn1_meth
Module: U:\extras\lib\libcrypto.lib(dsa_ameth.obj)
0001:00081d20  _dsa_asn1_meths
Module: U:\extras\lib\libcrypto.lib(ec_ameth.obj)
0001:00083270  _eckey_asn1_meth
Module: U:\extras\lib\libcrypto.lib(hm_ameth.obj)
0001:00083460  _hmac_asn1_meth
Module: U:\extras\lib\libcrypto.lib(a_dup.obj)
0001:000834c8  _ASN1_dup
0001:0008359c  _ASN1_item_dup
Module: U:\extras\lib\libcrypto.lib(asn_pack.obj)
0001:0008365b* _ASN1_seq_unpack
0001:000836d9* _ASN1_seq_pack
0001:000837ff* _ASN1_unpack_string
0001:00083864* _ASN1_pack_string
0001:000839a6  _ASN1_item_pack
0001:00083adb  _ASN1_item_unpack
Module: U:\extras\lib\libcrypto.lib(x_algor.obj)
0001:00083bb0  _X509_ALGOR_it
0001:00083c00  _X509_ALGORS_it
0001:00083c1c* _d2i_X509_ALGOR
0001:00083c45* _i2d_X509_ALGOR
0001:00083c67  _X509_ALGOR_new
0001:00083c7b  _X509_ALGOR_free
0001:00083c96* _d2i_X509_ALGORS
0001:00083cbf  _i2d_X509_ALGORS
0001:00083ce1* _X509_ALGOR_dup
0001:00083cfc  _X509_ALGOR_set0
0001:00083dbc  _X509_ALGOR_get0
Module: U:\extras\lib\libcrypto.lib(tb_cipher.obj)
0001:00083e10* _ENGINE_unregister_ciphers
0001:00083e3f* _ENGINE_register_ciphers
0001:00083eb7* _ENGINE_register_all_ciphers
0001:00083ee8* _ENGINE_set_default_ciphers
0001:00083f60  _ENGINE_get_cipher_engine
0001:00083f87  _ENGINE_get_cipher
0001:00083ffe* _ENGINE_get_ciphers
0001:00084009* _ENGINE_set_ciphers
Module: U:\extras\lib\libcrypto.lib(p12_utl.obj)
0001:0008402a  _OPENSSL_asc2uni
0001:000840e3* _OPENSSL_uni2asc
0001:00084173* _i2d_PKCS12_bio
0001:00084195* _i2d_PKCS12_fp
0001:000841b7* _d2i_PKCS12_bio
0001:000841d9* _d2i_PKCS12_fp
0001:000841fb* _PKCS12_x5092certbag
0001:00084226* _PKCS12_x509crl2certbag
0001:00084251* _PKCS12_certbag2x509
0001:000842ab* _PKCS12_certbag2x509crl
Module: U:\extras\lib\libcrypto.lib(x_bignum.obj)
0001:00084320  _BIGNUM_it
0001:00084340  _CBIGNUM_it
Module: U:\extras\lib\libcrypto.lib(x_long.obj)
0001:000844d0  _LONG_it
0001:00084500  _ZLONG_it
Module: U:\extras\lib\libcrypto.lib(rand_os2.obj)
0001:000847ab  _RAND_poll
Module: U:\extras\lib\libcrypto.lib(rsa_pk1.obj)
0001:00084b5a  _RSA_padding_add_PKCS1_type_1
0001:00084c0b  _RSA_padding_check_PKCS1_type_1
0001:00084dab  _RSA_padding_add_PKCS1_type_2
0001:00084ea3  _RSA_padding_check_PKCS1_type_2
Module: U:\extras\lib\libcrypto.lib(rsa_ssl.obj)
0001:0008501a  _RSA_padding_add_SSLv23
0001:00085134  _RSA_padding_check_SSLv23
Module: U:\extras\lib\libcrypto.lib(rsa_none.obj)
0001:0008530b  _RSA_padding_add_none
0001:000853a7  _RSA_padding_check_none
Module: U:\extras\lib\libcrypto.lib(bn_mod.obj)
0001:00085440  _BN_nnmod
0001:000854b8  _BN_mod_add
0001:00085504  _BN_mod_add_quick
0001:00085566* _BN_mod_sub
0001:000855b2  _BN_mod_sub_quick
0001:00085608  _BN_mod_mul
0001:000856c3  _BN_mod_sqr
0001:00085717* _BN_mod_lshift1
0001:0008575c  _BN_mod_lshift1_quick
0001:000857b7* _BN_mod_lshift
0001:0008586b  _BN_mod_lshift_quick
Module: U:\tmp\ldconv_libgcc_a_1a0352885a3d18ed28.lib(_alloca.obj)
0001:000859b0  __alloca
Module: U:\extras\lib\libcrypto.lib(bn_sqr.obj)
0001:000859e0  _BN_sqr
0001:00085c83* _bn_sqr_normal
0001:00085db2* _bn_sqr_recursive
Module: U:\extras\lib\libcrypto.lib(bn_recp.obj)
0001:00086060  _BN_RECP_CTX_init
0001:0008609f* _BN_RECP_CTX_new
0001:000860eb  _BN_RECP_CTX_free
0001:0008612d  _BN_RECP_CTX_set
0001:00086188  _BN_mod_mul_reciprocal
0001:00086258* _BN_div_recp
0001:00086583* _BN_reciprocal
Module: U:\extras\lib\libcrypto.lib(bn_exp2.obj)
0001:0008661a  _BN_mod_exp2_mont
Module: U:\extras\lib\libcrypto.lib(ech_ossl.obj)
0001:00086e14  _ECDH_OpenSSL
Module: U:\extras\lib\libcrypto.lib(tb_ecdh.obj)
0001:000872b4* _ENGINE_unregister_ECDH
0001:000872e3* _ENGINE_register_ECDH
0001:0008732f* _ENGINE_register_all_ECDH
0001:00087360* _ENGINE_set_default_ECDH
0001:000873ac  _ENGINE_get_default_ECDH
0001:000873c9  _ENGINE_get_ECDH
0001:000873d4* _ENGINE_set_ECDH
Module: U:\extras\lib\libcrypto.lib(ecp_nist.obj)
0001:000873f0  _EC_GFp_nist_method
0001:000873fa* _ec_GFp_nist_group_copy
0001:00087431* _ec_GFp_nist_group_set_curve
0001:000875d1* _ec_GFp_nist_field_mul
0001:000876bc* _ec_GFp_nist_field_sqr
Module: U:\extras\lib\libcrypto.lib(ecp_mont.obj)
0001:00087840  _EC_GFp_mont_method
0001:0008784a* _ec_GFp_mont_group_init
0001:0008787d* _ec_GFp_mont_group_finish
0001:000878e6* _ec_GFp_mont_group_clear_finish
0001:0008794f* _ec_GFp_mont_group_copy
0001:00087a9d* _ec_GFp_mont_group_set_curve
0001:00087ca6* _ec_GFp_mont_field_mul
0001:00087d1b* _ec_GFp_mont_field_sqr
0001:00087d90* _ec_GFp_mont_field_encode
0001:00087e0e* _ec_GFp_mont_field_decode
0001:00087e7c* _ec_GFp_mont_field_set_to_one
Module: U:\extras\lib\libcrypto.lib(ec2_smpl.obj)
0001:00087f90  _EC_GF2m_simple_method
0001:00087f9a* _ec_GF2m_simple_group_init
0001:00087fd3* _ec_GF2m_simple_group_finish
0001:00088007* _ec_GF2m_simple_group_clear_finish
0001:00088077* _ec_GF2m_simple_group_copy
0001:0008827e  _ec_GF2m_simple_group_set_curve
0001:00088498* _ec_GF2m_simple_group_get_curve
0001:0008851d* _ec_GF2m_simple_group_get_degree
0001:00088534* _ec_GF2m_simple_group_check_discriminant
0001:00088615* _ec_GF2m_simple_point_init
0001:0008864c* _ec_GF2m_simple_point_finish
0001:0008867e* _ec_GF2m_simple_point_clear_finish
0001:000886ba* _ec_GF2m_simple_point_copy
0001:0008873c* _ec_GF2m_simple_point_set_to_infinity
0001:00088769* _ec_GF2m_simple_point_set_affine_coordinates
0001:0008886a* _ec_GF2m_simple_point_get_affine_coordinates
0001:00088987* _ec_GF2m_simple_set_compressed_coordinates
0001:00088cd4* _ec_GF2m_simple_point2oct
0001:0008911f* _ec_GF2m_simple_oct2point
0001:000895a6* _ec_GF2m_simple_add
0001:00089b37* _ec_GF2m_simple_dbl
0001:00089b66* _ec_GF2m_simple_invert
0001:00089bdb* _ec_GF2m_simple_is_at_infinity
0001:00089bee* _ec_GF2m_simple_is_on_curve
0001:00089e0c* _ec_GF2m_simple_cmp
0001:0008a004* _ec_GF2m_simple_make_affine
0001:0008a14b* _ec_GF2m_simple_points_make_affine
0001:0008a19d* _ec_GF2m_simple_field_mul
0001:0008a1cf* _ec_GF2m_simple_field_sqr
0001:0008a1fa* _ec_GF2m_simple_field_div
Module: U:\extras\lib\libcrypto.lib(x509_v3.obj)
0001:0008a2d0  _X509v3_get_ext_count
0001:0008a2f0  _X509v3_get_ext_by_NID
0001:0008a32c  _X509v3_get_ext_by_OBJ
0001:0008a3a3  _X509v3_get_ext_by_critical
0001:0008a422  _X509v3_get_ext
0001:0008a45f  _X509v3_delete_ext
0001:0008a4ac  _X509v3_add_ext
0001:0008a5e2  _X509_EXTENSION_create_by_NID
0001:0008a668  _X509_EXTENSION_create_by_OBJ
0001:0008a753* _X509_EXTENSION_set_object
0001:0008a790* _X509_EXTENSION_set_critical
0001:0008a7bf* _X509_EXTENSION_set_data
0001:0008a80a  _X509_EXTENSION_get_object
0001:0008a821  _X509_EXTENSION_get_data
0001:0008a839  _X509_EXTENSION_get_critical
Module: U:\extras\lib\libcrypto.lib(x509_obj.obj)
0001:0008a888  _X509_NAME_oneline
Module: U:\extras\lib\libcrypto.lib(v3_purp.obj)
0001:0008add1  _X509_check_purpose
0001:0008afaa  _X509_PURPOSE_get_by_id
0001:0008af0d  _X509_PURPOSE_get0
0001:0008ae8d  _X509_PURPOSE_set
0001:0008aee5* _X509_PURPOSE_get_count
0001:0008af5b* _X509_PURPOSE_get_by_sname
0001:0008b004* _X509_PURPOSE_add
0001:0008b27a* _X509_PURPOSE_cleanup
0001:0008b2d4* _X509_PURPOSE_get_id
0001:0008b2de* _X509_PURPOSE_get0_name
0001:0008b2e9* _X509_PURPOSE_get0_sname
0001:0008b2f4* _X509_PURPOSE_get_trust
0001:0008b36b* _X509_supported_extension
0001:0008bc5b  _X509_check_ca
0001:0008c108  _X509_check_issued
0001:0008c1e2  _X509_check_akid
Module: U:\extras\lib\libcrypto.lib(x_name.obj)
0001:0008c410  _X509_NAME_ENTRY_it
0001:0008c42c* _d2i_X509_NAME_ENTRY
0001:0008c455* _i2d_X509_NAME_ENTRY
0001:0008c477  _X509_NAME_ENTRY_new
0001:0008c48b  _X509_NAME_ENTRY_free
0001:0008c4a6  _X509_NAME_ENTRY_dup
0001:0008c500* _X509_NAME_ENTRIES_it
0001:0008c560* _X509_NAME_INTERNAL_it
0001:0008c580* _x509_name_ff
0001:0008c5b0  _X509_NAME_it
0001:0008c5cc* _d2i_X509_NAME
0001:0008c5f5  _i2d_X509_NAME
0001:0008c617  _X509_NAME_new
0001:0008c62b  _X509_NAME_free
0001:0008c646  _X509_NAME_dup
0001:0008d108  _X509_NAME_set
Module: U:\extras\lib\libcrypto.lib(x_pubkey.obj)
0001:0008d210  _X509_PUBKEY_it
0001:0008d22c* _d2i_X509_PUBKEY
0001:0008d255* _i2d_X509_PUBKEY
0001:0008d277* _X509_PUBKEY_new
0001:0008d28b* _X509_PUBKEY_free
0001:0008d2b1  _X509_PUBKEY_set
0001:0008d3e6  _X509_PUBKEY_get
0001:0008d5c0  _d2i_PUBKEY
0001:0008d636  _i2d_PUBKEY
0001:0008d692  _d2i_RSA_PUBKEY
0001:0008d718  _i2d_RSA_PUBKEY
0001:0008d7a3  _d2i_DSA_PUBKEY
0001:0008d829  _i2d_DSA_PUBKEY
0001:0008d8b4  _d2i_EC_PUBKEY
0001:0008d93a  _i2d_EC_PUBKEY
0001:0008d9c5  _X509_PUBKEY_set0_param
0001:0008da64  _X509_PUBKEY_get0_param
Module: U:\extras\lib\libcrypto.lib(v3_alt.obj)
0001:0008dac0  _v3_alt
0001:0008db68  _i2v_GENERAL_NAMES
0001:0008dc45  _i2v_GENERAL_NAME
0001:0008dfd0  _GENERAL_NAME_print
0001:0008e979  _v2i_GENERAL_NAME
0001:0008e8a2  _v2i_GENERAL_NAMES
0001:0008ed25  _v2i_GENERAL_NAME_ex
0001:0008e9b1* _a2i_GENERAL_NAME
Module: U:\extras\lib\libcrypto.lib(x_req.obj)
0001:0008f1e0  _X509_REQ_INFO_it
0001:0008f1fc* _d2i_X509_REQ_INFO
0001:0008f225* _i2d_X509_REQ_INFO
0001:0008f247* _X509_REQ_INFO_new
0001:0008f25b* _X509_REQ_INFO_free
0001:0008f310  _X509_REQ_it
0001:0008f32c* _d2i_X509_REQ
0001:0008f355* _i2d_X509_REQ
0001:0008f377  _X509_REQ_new
0001:0008f38b  _X509_REQ_free
0001:0008f3a6* _X509_REQ_dup
Module: U:\extras\lib\libcrypto.lib(x509rset.obj)
0001:0008f3d0* _X509_REQ_set_version
0001:0008f3fc  _X509_REQ_set_subject_name
0001:0008f431  _X509_REQ_set_pubkey
Module: U:\extras\lib\libcrypto.lib(x_all.obj)
0001:0008f470  _X509_verify
0001:0008f4ad* _X509_REQ_verify
0001:0008f4ea* _NETSCAPE_SPKI_verify
0001:0008f527* _X509_sign
0001:0008f585  _X509_REQ_sign
0001:0008f5d1* _X509_CRL_sign
0001:0008f62f* _NETSCAPE_SPKI_sign
0001:0008f67b* _d2i_X509_fp
0001:0008f69d* _i2d_X509_fp
0001:0008f6bf* _d2i_X509_bio
0001:0008f6e1* _i2d_X509_bio
0001:0008f703* _d2i_X509_CRL_fp
0001:0008f725* _i2d_X509_CRL_fp
0001:0008f747* _d2i_X509_CRL_bio
0001:0008f769* _i2d_X509_CRL_bio
0001:0008f78b* _d2i_PKCS7_fp
0001:0008f7ad* _i2d_PKCS7_fp
0001:0008f7cf* _d2i_PKCS7_bio
0001:0008f7f1* _i2d_PKCS7_bio
0001:0008f813* _d2i_X509_REQ_fp
0001:0008f835* _i2d_X509_REQ_fp
0001:0008f857* _d2i_X509_REQ_bio
0001:0008f879* _i2d_X509_REQ_bio
0001:0008f89b* _d2i_RSAPrivateKey_fp
0001:0008f8bd* _i2d_RSAPrivateKey_fp
0001:0008f8df* _d2i_RSAPublicKey_fp
0001:0008f901* _d2i_RSA_PUBKEY_fp
0001:0008f92d* _i2d_RSAPublicKey_fp
0001:0008f94f* _i2d_RSA_PUBKEY_fp
0001:0008f972* _d2i_RSAPrivateKey_bio
0001:0008f994* _i2d_RSAPrivateKey_bio
0001:0008f9b6* _d2i_RSAPublicKey_bio
0001:0008f9d8* _d2i_RSA_PUBKEY_bio
0001:0008fa04* _i2d_RSAPublicKey_bio
0001:0008fa26* _i2d_RSA_PUBKEY_bio
0001:0008fa49* _d2i_DSAPrivateKey_fp
0001:0008fa75* _i2d_DSAPrivateKey_fp
0001:0008fa98* _d2i_DSA_PUBKEY_fp
0001:0008fac4* _i2d_DSA_PUBKEY_fp
0001:0008fae7* _d2i_DSAPrivateKey_bio
0001:0008fb13* _i2d_DSAPrivateKey_bio
0001:0008fb36* _d2i_DSA_PUBKEY_bio
0001:0008fb62* _i2d_DSA_PUBKEY_bio
0001:0008fb85* _d2i_EC_PUBKEY_fp
0001:0008fbb1* _i2d_EC_PUBKEY_fp
0001:0008fbd4* _d2i_ECPrivateKey_fp
0001:0008fc00* _i2d_ECPrivateKey_fp
0001:0008fc23* _d2i_EC_PUBKEY_bio
0001:0008fc4f* _i2d_EC_PUBKEY_bio
0001:0008fc72* _d2i_ECPrivateKey_bio
0001:0008fc9e* _i2d_ECPrivateKey_bio
0001:0008fcc1* _X509_pubkey_digest
0001:0008fd1a  _X509_digest
0001:0008fd4a  _X509_CRL_digest
0001:0008fd7a* _X509_REQ_digest
0001:0008fdaa* _X509_NAME_digest
0001:0008fdda* _PKCS7_ISSUER_AND_SERIAL_digest
0001:0008fe0a* _d2i_PKCS8_fp
0001:0008fe36* _i2d_PKCS8_fp
0001:0008fe59* _d2i_PKCS8_bio
0001:0008fe85* _i2d_PKCS8_bio
0001:0008fea8* _d2i_PKCS8_PRIV_KEY_INFO_fp
0001:0008fed4* _i2d_PKCS8_PRIV_KEY_INFO_fp
0001:0008fef7* _i2d_PKCS8PrivateKeyInfo_fp
0001:0008ff3d* _i2d_PrivateKey_fp
0001:0008ff60* _d2i_PrivateKey_fp
0001:0008ff8c* _i2d_PUBKEY_fp
0001:0008ffaf* _d2i_PUBKEY_fp
0001:0008ffdb* _d2i_PKCS8_PRIV_KEY_INFO_bio
0001:00090007* _i2d_PKCS8_PRIV_KEY_INFO_bio
0001:0009002a* _i2d_PKCS8PrivateKeyInfo_bio
0001:00090070* _i2d_PrivateKey_bio
0001:00090093* _d2i_PrivateKey_bio
0001:000900bf* _i2d_PUBKEY_bio
0001:000900e2* _d2i_PUBKEY_bio
Module: U:\extras\lib\libcrypto.lib(x509_att.obj)
0001:00090110  _X509at_get_attr_count
0001:00090123  _X509at_get_attr_by_NID
0001:0009015f  _X509at_get_attr_by_OBJ
0001:000901d6  _X509at_get_attr
0001:00090213  _X509at_delete_attr
0001:00090261  _X509at_add1_attr
0001:00090366  _X509at_add1_attr_by_OBJ
0001:000905cc* _X509_ATTRIBUTE_create_by_OBJ
0001:000903c9  _X509at_add1_attr_by_NID
0001:0009053f* _X509_ATTRIBUTE_create_by_NID
0001:0009042c  _X509at_add1_attr_by_txt
0001:000906b2* _X509_ATTRIBUTE_create_by_txt
0001:0009048f  _X509at_get0_data_by_OBJ
0001:0009097a* _X509_ATTRIBUTE_count
0001:000909c9* _X509_ATTRIBUTE_get0_data
0001:0009075c* _X509_ATTRIBUTE_set1_object
0001:00090799* _X509_ATTRIBUTE_set1_data
0001:000909b2* _X509_ATTRIBUTE_get0_object
0001:00090a3c* _X509_ATTRIBUTE_get0_type
Module: U:\extras\lib\libcrypto.lib(v3_bitst.obj)
0001:00090c30  _v3_nscert
0001:00090ca8* _i2v_ASN1_BIT_STRING
0001:00090d24* _v2i_ASN1_BIT_STRING
0001:00090c70  _v3_key_usage
Module: U:\extras\lib\libcrypto.lib(v3_ia5.obj)
0001:00090f00  _v3_ns_ia5_list
Module: U:\extras\lib\libcrypto.lib(v3_skey.obj)
0001:00091240  _v3_skey_id
0001:00091278* _i2s_ASN1_OCTET_STRING
0001:000912a1* _s2i_ASN1_OCTET_STRING
Module: U:\extras\lib\libcrypto.lib(v3_pku.obj)
0001:00091520  _v3_pkey_usage_period
0001:000915b0* _PKEY_USAGE_PERIOD_it
0001:000915cc* _d2i_PKEY_USAGE_PERIOD
0001:000915f5* _i2d_PKEY_USAGE_PERIOD
0001:00091617* _PKEY_USAGE_PERIOD_new
0001:0009162b* _PKEY_USAGE_PERIOD_free
Module: U:\extras\lib\libcrypto.lib(v3_bcons.obj)
0001:00091730  _v3_bcons
0001:000917c0* _BASIC_CONSTRAINTS_it
0001:000917dc* _d2i_BASIC_CONSTRAINTS
0001:00091805* _i2d_BASIC_CONSTRAINTS
0001:00091827* _BASIC_CONSTRAINTS_new
0001:0009183b  _BASIC_CONSTRAINTS_free
Module: U:\extras\lib\libcrypto.lib(v3_int.obj)
0001:00091a40  _v3_crl_num
0001:00091a80  _v3_delta_crl
0001:00091ae0  _v3_inhibit_anyp
Module: U:\extras\lib\libcrypto.lib(v3_cpols.obj)
0001:00091b20  _v3_cpols
0001:00091b90* _CERTIFICATEPOLICIES_it
0001:00091c80* _POLICYINFO_it
0001:00091bac* _d2i_CERTIFICATEPOLICIES
0001:00091bd5* _i2d_CERTIFICATEPOLICIES
0001:00091bf7* _CERTIFICATEPOLICIES_new
0001:00091c0b* _CERTIFICATEPOLICIES_free
0001:00091df0* _POLICYQUALINFO_it
0001:00091c9c* _d2i_POLICYINFO
0001:00091cc5* _i2d_POLICYINFO
0001:00091ce7* _POLICYINFO_new
0001:00091cfb  _POLICYINFO_free
0001:00091ee0* _USERNOTICE_it
0001:00091e0c* _d2i_POLICYQUALINFO
0001:00091e35* _i2d_POLICYQUALINFO
0001:00091e57* _POLICYQUALINFO_new
0001:00091e6b  _POLICYQUALINFO_free
0001:00091fd0* _NOTICEREF_it
0001:00091efc* _d2i_USERNOTICE
0001:00091f25* _i2d_USERNOTICE
0001:00091f47* _USERNOTICE_new
0001:00091f5b* _USERNOTICE_free
0001:00091fec* _d2i_NOTICEREF
0001:00092015* _i2d_NOTICEREF
0001:00092037* _NOTICEREF_new
0001:0009204b* _NOTICEREF_free
0001:0009313c* _X509_POLICY_NODE_print
Module: U:\extras\lib\libcrypto.lib(v3_akey.obj)
0001:00093230  _v3_akey_id
Module: U:\extras\lib\libcrypto.lib(v3_crld.obj)
0001:00093710  _v3_crld
0001:00094480* _CRL_DIST_POINTS_it
0001:00093750  _v3_freshest_crl
0001:00094317* _DIST_POINT_NAME_new
0001:00094407* _DIST_POINT_new
0001:0009441b* _DIST_POINT_free
0001:000942b0* _DIST_POINT_NAME_it
0001:000942cc* _d2i_DIST_POINT_NAME
0001:000942f5* _i2d_DIST_POINT_NAME
0001:0009432b* _DIST_POINT_NAME_free
0001:000943a0* _DIST_POINT_it
0001:000943bc* _d2i_DIST_POINT
0001:000943e5* _i2d_DIST_POINT
0001:0009449c* _d2i_CRL_DIST_POINTS
0001:000944c5* _i2d_CRL_DIST_POINTS
0001:000944e7* _CRL_DIST_POINTS_new
0001:000944fb  _CRL_DIST_POINTS_free
0001:000945e0* _ISSUING_DIST_POINT_it
0001:000945fc* _d2i_ISSUING_DIST_POINT
0001:00094625* _i2d_ISSUING_DIST_POINT
0001:00094647* _ISSUING_DIST_POINT_new
0001:0009465b  _ISSUING_DIST_POINT_free
0001:00094680  _v3_idp
0001:00094dba  _DIST_POINT_set_dpname
Module: U:\extras\lib\libcrypto.lib(v3_extku.obj)
0001:00094ed0  _v3_ext_ku
0001:00094f80* _EXTENDED_KEY_USAGE_it
0001:00094f10  _v3_ocsp_accresp
0001:00094f9c* _d2i_EXTENDED_KEY_USAGE
0001:00094fc5* _i2d_EXTENDED_KEY_USAGE
0001:00094fe7* _EXTENDED_KEY_USAGE_new
0001:00094ffb* _EXTENDED_KEY_USAGE_free
Module: U:\extras\lib\libcrypto.lib(v3_enum.obj)
0001:00095350  _v3_crl_reason
0001:00095388* _i2s_ASN1_ENUMERATED_TABLE
Module: U:\extras\lib\libcrypto.lib(v3_ocsp.obj)
0001:000953f0  _v3_ocsp_crlid
0001:00095430  _v3_ocsp_acutoff
0001:00095470  _v3_crl_invdate
0001:000954b0  _v3_crl_hold
0001:000954f0  _v3_ocsp_nonce
0001:00095530  _v3_ocsp_nocheck
0001:00095570  _v3_ocsp_serviceloc
Module: U:\extras\lib\libcrypto.lib(v3_sxnet.obj)
0001:00095b00  _v3_sxnet
0001:00095c60* _SXNET_it
0001:00095b80* _SXNETID_it
0001:00095b9c* _d2i_SXNETID
0001:00095bc5* _i2d_SXNETID
0001:00095be7* _SXNETID_new
0001:00095bfb* _SXNETID_free
0001:00095c7c* _d2i_SXNET
0001:00095ca5* _i2d_SXNET
0001:00095cc7* _SXNET_new
0001:00095cdb* _SXNET_free
0001:00095e90* _SXNET_add_id_asc
0001:00095fa6* _SXNET_add_id_INTEGER
0001:00095f0e* _SXNET_add_id_ulong
0001:000962cd* _SXNET_get_id_INTEGER
0001:000961b1* _SXNET_get_id_asc
0001:00096232* _SXNET_get_id_ulong
Module: U:\extras\lib\libcrypto.lib(v3_pcons.obj)
0001:00096340  _v3_policy_constraints
0001:000963f0* _POLICY_CONSTRAINTS_it
0001:0009640c* _POLICY_CONSTRAINTS_new
0001:00096420  _POLICY_CONSTRAINTS_free
Module: U:\extras\lib\libcrypto.lib(v3_pci.obj)
0001:000966a0  _v3_pci
Module: U:\extras\lib\libcrypto.lib(v3_ncons.obj)
0001:00097670  _v3_name_constraints
0001:00097790* _NAME_CONSTRAINTS_it
0001:00097710* _GENERAL_SUBTREE_it
0001:000977ac* _GENERAL_SUBTREE_new
0001:000977c0* _GENERAL_SUBTREE_free
0001:000977db* _NAME_CONSTRAINTS_new
0001:000977ef  _NAME_CONSTRAINTS_free
0001:00097d48  _NAME_CONSTRAINTS_check
Module: U:\extras\lib\libcrypto.lib(v3_pmaps.obj)
0001:00098440  _v3_policy_mappings
0001:00098530* _POLICY_MAPPINGS_it
0001:000984e0* _POLICY_MAPPING_it
0001:0009854c* _POLICY_MAPPING_new
0001:00098560  _POLICY_MAPPING_free
Module: U:\extras\lib\libcrypto.lib(v3_conf.obj)
0001:00098921* _X509V3_EXT_nconf
0001:00098a0d* _X509V3_EXT_nconf_nid
0001:00098ecf  _X509V3_EXT_i2d
0001:000992ad* _X509V3_EXT_add_nconf_sk
0001:00099375* _X509V3_EXT_add_nconf
0001:000993b5* _X509V3_EXT_CRL_add_nconf
0001:000993f5* _X509V3_EXT_REQ_add_nconf
0001:00099477* _X509V3_get_string
0001:00099506  _X509V3_get_section
0001:00099591* _X509V3_string_free
0001:000995ca  _X509V3_section_free
0001:0009963e  _X509V3_set_nconf
0001:00099656* _X509V3_set_ctx
0001:00099687* _X509V3_EXT_conf
0001:000996c1* _X509V3_EXT_conf_nid
0001:00099736* _X509V3_set_conf_lhash
0001:0009974e* _X509V3_EXT_add_conf
0001:00099788* _X509V3_EXT_CRL_add_conf
0001:000997c2* _X509V3_EXT_REQ_add_conf
Module: U:\extras\lib\libcrypto.lib(a_strnid.obj)
0001:00099800* _ASN1_STRING_set_default_mask
0001:0009980d* _ASN1_STRING_get_default_mask
0001:0009983b* _ASN1_STRING_set_default_mask_asc
0001:00099946  _ASN1_STRING_set_by_NID
0001:00099c21* _ASN1_STRING_TABLE_get
0001:00099cab* _ASN1_STRING_TABLE_add
0001:00099df7* _ASN1_STRING_TABLE_cleanup
Module: U:\extras\lib\libcrypto.lib(a_print.obj)
0001:00099e50  _ASN1_PRINTABLE_type
0001:00099f5e* _ASN1_UNIVERSALSTRING_to_string
Module: U:\extras\lib\libcrypto.lib(conf_lib.obj)
0001:0009a060* _CONF_version
0001:0009a088  _CONF_set_nconf
0001:0009a0bc* _CONF_set_default_method
0001:0009a0dc* _CONF_load
0001:0009a1e5* _CONF_load_bio
0001:0009a164* _CONF_load_fp
0001:0009a587* _NCONF_load_bio
0001:0009a22b  _CONF_get_section
0001:0009a5e6  _NCONF_get_section
0001:0009a264  _CONF_get_string
0001:0009a680  _NCONF_get_string
0001:0009a2b9* _CONF_get_number
0001:0009a746* _NCONF_get_number_e
0001:0009a337  _CONF_free
0001:0009a486* _NCONF_free_data
0001:0009a35c* _CONF_dump_fp
0001:0009a3d6* _CONF_dump_bio
0001:0009a899* _NCONF_dump_bio
0001:0009a402  _NCONF_new
0001:0009a465  _NCONF_free
0001:0009a4a7  _NCONF_load
0001:0009a506* _NCONF_load_fp
0001:0009a81f* _NCONF_dump_fp
Module: U:\extras\lib\libcrypto.lib(dso_lib.obj)
0001:0009a900* _DSO_new
0001:0009a95a* _DSO_new_method
0001:0009a914* _DSO_set_default_method
0001:0009a921* _DSO_get_default_method
0001:0009a92b* _DSO_get_method
0001:0009a935* _DSO_set_method
0001:0009aa9a  _DSO_free
0001:0009ac16* _DSO_flags
0001:0009ac2e* _DSO_up_ref
0001:0009aca2  _DSO_load
0001:0009b08f* _DSO_ctrl
0001:0009b22f* _DSO_set_filename
0001:0009aec3* _DSO_bind_var
0001:0009afa9  _DSO_bind_func
0001:0009b188* _DSO_set_name_converter
0001:0009b1e8* _DSO_get_filename
0001:0009b361* _DSO_merge
0001:0009b417* _DSO_convert_filename
0001:0009b593* _DSO_get_loaded_filename
0001:0009b5da* _DSO_pathbyaddr
0001:0009b651* _DSO_global_lookup
Module: U:\extras\lib\libcrypto.lib(x509_def.obj)
0001:0009b6d0* _X509_get_default_private_dir
0001:0009b6e2  _X509_get_default_cert_area
0001:0009b6fa* _X509_get_default_cert_dir
0001:0009b715* _X509_get_default_cert_file
0001:0009b72c* _X509_get_default_cert_dir_env
0001:0009b744* _X509_get_default_cert_file_env
Module: U:\extras\lib\libcrypto.lib(rsa_asn1.obj)
0001:0009b8b0  _RSAPrivateKey_it
0001:0009b920  _RSAPublicKey_it
0001:0009b93c  _d2i_RSAPrivateKey
0001:0009b965  _i2d_RSAPrivateKey
0001:0009b987  _d2i_RSAPublicKey
0001:0009b9b0  _i2d_RSAPublicKey
0001:0009b9d2* _RSAPublicKey_dup
0001:0009b9ed* _RSAPrivateKey_dup
Module: U:\extras\lib\libcrypto.lib(p8_pkey.obj)
0001:0009bb10  _PKCS8_PRIV_KEY_INFO_it
0001:0009bb2c  _d2i_PKCS8_PRIV_KEY_INFO
0001:0009bb55  _i2d_PKCS8_PRIV_KEY_INFO
0001:0009bb77  _PKCS8_PRIV_KEY_INFO_new
0001:0009bb8b  _PKCS8_PRIV_KEY_INFO_free
0001:0009bba6  _PKCS8_pkey_set0
0001:0009bc8e  _PKCS8_pkey_get0
Module: U:\extras\lib\libcrypto.lib(t_pkey.obj)
0001:0009bd89  _ASN1_bn_print
Module: U:\extras\lib\libcrypto.lib(pk7_lib.obj)
0001:0009bfda  _PKCS7_ctrl
0001:0009c15b* _PKCS7_content_new
0001:0009c281  _PKCS7_set_type
0001:0009c1c8* _PKCS7_set_content
0001:0009c51d* _PKCS7_set0_type_other
0001:0009c544* _PKCS7_add_signer
0001:0009c70d* _PKCS7_add_certificate
0001:0009c835* _PKCS7_add_crl
0001:0009c95d* _PKCS7_SIGNER_INFO_set
0001:0009cb12* _PKCS7_add_signature
0001:0009cbf8* _PKCS7_set_digest
0001:0009cccf* _PKCS7_get_signer_info
0001:0009cd18  _PKCS7_SIGNER_INFO_get0_algs
0001:0009cd50  _PKCS7_RECIP_INFO_get0_alg
0001:0009cd66* _PKCS7_add_recipient
0001:0009ce61* _PKCS7_RECIP_INFO_set
0001:0009cdca* _PKCS7_add_recipient_info
0001:0009d04f* _PKCS7_cert_from_signer_info
0001:0009d09b* _PKCS7_set_cipher
0001:0009d165  _PKCS7_stream
Module: U:\extras\lib\libcrypto.lib(cms_sd.obj)
0001:0009d39c* _CMS_SignedData_init
0001:0009df6a* _CMS_get0_SignerInfos
0001:0009d6cf  _cms_set1_SignerIdentifier
0001:0009d837  _cms_SignerIdentifier_get0_signer_id
0001:0009d897  _cms_SignerIdentifier_cert_cmp
0001:0009d94c* _CMS_add1_signer
0001:0009ee9f* _CMS_add_standard_smimecap
0001:0009ecc1* _CMS_add_smimecap
0001:0009e572* _CMS_SignerInfo_sign
0001:0009df93* _CMS_get0_signers
0001:0009e034* _CMS_SignerInfo_set1_signer_cert
0001:0009e0ba* _CMS_SignerInfo_get0_signer_id
0001:0009e0e5* _CMS_SignerInfo_cert_cmp
0001:0009e102* _CMS_set1_signers_certs
0001:0009e277  _CMS_SignerInfo_get0_algs
0001:0009e4f2  _cms_SignedData_final
0001:0009e826* _CMS_SignerInfo_verify
0001:0009e9c4  _cms_SignedData_init_bio
0001:0009ea93* _CMS_SignerInfo_verify_content
0001:0009ed2c* _CMS_add_simple_smimecap
Module: U:\extras\lib\libcrypto.lib(cms_env.obj)
0001:0009f11d* _CMS_get0_RecipientInfos
0001:0009f146* _CMS_RecipientInfo_type
0001:0009f150* _CMS_EnvelopedData_create
0001:0009f1f1* _CMS_add1_recipient_cert
0001:0009f488  _CMS_RecipientInfo_ktri_get0_algs
0001:0009f50d* _CMS_RecipientInfo_ktri_get0_signer_id
0001:0009f57d* _CMS_RecipientInfo_ktri_cert_cmp
0001:0009f5d9* _CMS_RecipientInfo_set0_pkey
0001:0009faac* _CMS_RecipientInfo_kekri_id_cmp
0001:0009fb62* _CMS_add0_recipient_key
0001:0009fe08* _CMS_RecipientInfo_kekri_get0_id
0001:0009fee7* _CMS_RecipientInfo_set0_key
0001:000a03a7* _CMS_RecipientInfo_decrypt
0001:000a0418  _cms_EnvelopedData_init_bio
Module: U:\extras\lib\libcrypto.lib(dh_asn1.obj)
0001:000a0680* _DHparams_it
0001:000a069c  _d2i_DHparams
0001:000a06c5  _i2d_DHparams
0001:000a06e7* _DHparams_dup
Module: U:\extras\lib\libcrypto.lib(ec_asn1.obj)
0001:000a0710  _EC_GROUP_get_basis_type
0001:000a0780* _EC_GROUP_get_trinomial_basis
0001:000a0813* _EC_GROUP_get_pentanomial_basis
0001:000a0940* _X9_62_PENTANOMIAL_it
0001:000a095c* _X9_62_PENTANOMIAL_new
0001:000a0970* _X9_62_PENTANOMIAL_free
0001:000a0ab0* _X9_62_CHARACTERISTIC_TWO_it
0001:000a0acc* _X9_62_CHARACTERISTIC_TWO_new
0001:000a0ae0* _X9_62_CHARACTERISTIC_TWO_free
0001:000a0bd0* _X9_62_FIELDID_it
0001:000a0c50* _X9_62_CURVE_it
0001:000a0d30* _ECPARAMETERS_it
0001:000a0d4c* _ECPARAMETERS_new
0001:000a0d60* _ECPARAMETERS_free
0001:000a0e10* _ECPKPARAMETERS_it
0001:000a0e2c* _d2i_UC_ECPKPARAMETERS
0001:000a0e55* _i2d_UC_ECPKPARAMETERS
0001:000a0e77* _ECPKPARAMETERS_new
0001:000a0e8b* _ECPKPARAMETERS_free
0001:000a0f30* _EC_PRIVATEKEY_it
0001:000a0f4c* _d2i_EC_PRIVATEKEY
0001:000a0f75* _i2d_EC_PRIVATEKEY
0001:000a0f97* _EC_PRIVATEKEY_new
0001:000a0fab* _EC_PRIVATEKEY_free
0001:000a2bac* _d2i_ECPKParameters
0001:000a2ca2* _i2d_ECPKParameters
0001:000a2d67  _d2i_ECPrivateKey
0001:000a30ed  _i2d_ECPrivateKey
0001:000a3597  _i2d_ECParameters
0001:000a35ed  _d2i_ECParameters
0001:000a36fb  _o2i_ECPublicKey
0001:000a3854  _i2o_ECPublicKey
Module: U:\extras\lib\libcrypto.lib(ec_print.obj)
0001:000a3a1b  _EC_POINT_point2bn
0001:000a3b06* _EC_POINT_bn2point
0001:000a3c38* _EC_POINT_point2hex
0001:000a3da7* _EC_POINT_hex2point
Module: U:\extras\lib\libcrypto.lib(eck_prn.obj)
0001:000a3e1a* _ECPKParameters_print_fp
0001:000a411c  _ECPKParameters_print
0001:000a3eb7* _EC_KEY_print_fp
0001:000a3fea* _EC_KEY_print
0001:000a3f54* _ECParameters_print_fp
0001:000a404f* _ECParameters_print
Module: U:\extras\lib\libcrypto.lib(a_set.obj)
0001:000a4b5c  _i2d_ASN1_SET
0001:000a4e87  _d2i_ASN1_SET
Module: U:\extras\lib\libcrypto.lib(p12_asn.obj)
0001:000a52e0* _PKCS12_MAC_DATA_it
0001:000a51e0  _PKCS12_it
0001:000a51fc* _d2i_PKCS12
0001:000a5225* _i2d_PKCS12
0001:000a5247* _PKCS12_new
0001:000a525b* _PKCS12_free
0001:000a52fc* _d2i_PKCS12_MAC_DATA
0001:000a5325* _i2d_PKCS12_MAC_DATA
0001:000a5347* _PKCS12_MAC_DATA_new
0001:000a535b* _PKCS12_MAC_DATA_free
0001:000a5480* _PKCS12_BAGS_it
0001:000a549c* _d2i_PKCS12_BAGS
0001:000a54c5* _i2d_PKCS12_BAGS
0001:000a54e7  _PKCS12_BAGS_new
0001:000a54fb* _PKCS12_BAGS_free
0001:000a5680* _PKCS12_SAFEBAG_it
0001:000a569c* _d2i_PKCS12_SAFEBAG
0001:000a56c5* _i2d_PKCS12_SAFEBAG
0001:000a56e7  _PKCS12_SAFEBAG_new
0001:000a56fb* _PKCS12_SAFEBAG_free
0001:000a5750  _PKCS12_SAFEBAGS_it
0001:000a57a0  _PKCS12_AUTHSAFES_it
Module: U:\extras\lib\libcrypto.lib(a_i2d_fp.obj)
0001:000a57cb  _ASN1_i2d_fp
0001:000a5868  _ASN1_i2d_bio
0001:000a5956  _ASN1_item_i2d_fp
0001:000a59f3  _ASN1_item_i2d_bio
Module: U:\extras\lib\libcrypto.lib(a_d2i_fp.obj)
0001:000a5acb  _ASN1_d2i_fp
0001:000a5b6f  _ASN1_d2i_bio
0001:000a5bdd  _ASN1_item_d2i_bio
0001:000a5c52  _ASN1_item_d2i_fp
Module: U:\extras\lib\libcrypto.lib(x_x509.obj)
0001:000a61b0  _X509_CINF_it
0001:000a61cc* _d2i_X509_CINF
0001:000a61f5* _i2d_X509_CINF
0001:000a6217* _X509_CINF_new
0001:000a622b* _X509_CINF_free
0001:000a6450  _X509_it
0001:000a646c* _d2i_X509
0001:000a6495* _i2d_X509
0001:000a64b7* _X509_new
0001:000a64cb  _X509_free
0001:000a64e6* _X509_dup
0001:000a6501* _X509_get_ex_new_index
0001:000a6538* _X509_set_ex_data
0001:000a655c* _X509_get_ex_data
0001:000a6579* _d2i_X509_AUX
0001:000a6604* _i2d_X509_AUX
Module: U:\extras\lib\libcrypto.lib(p12_add.obj)
0001:000a665a  _PKCS12_item_pack_safebag
0001:000a6766* _PKCS12_MAKE_KEYBAG
0001:000a67cc* _PKCS12_MAKE_SHKEYBAG
0001:000a68ce* _PKCS12_pack_p7data
0001:000a69d2* _PKCS12_unpack_p7data
0001:000a6a36* _PKCS12_pack_p7encdata
0001:000a6c24* _PKCS12_unpack_p7encdata
0001:000a6c88* _PKCS12_decrypt_skey
0001:000a6cac* _PKCS12_pack_authsafes
0001:000a6ce4* _PKCS12_unpack_authsafes
Module: U:\extras\lib\libcrypto.lib(x_crl.obj)
0001:000a6dd0* _X509_REVOKED_it
0001:000a6f30  _X509_CRL_INFO_it
0001:000a7630  _X509_CRL_it
0001:000a764c* _d2i_X509_REVOKED
0001:000a7675* _i2d_X509_REVOKED
0001:000a7697* _X509_REVOKED_new
0001:000a76ab* _X509_REVOKED_free
0001:000a76c6* _d2i_X509_CRL_INFO
0001:000a76ef* _i2d_X509_CRL_INFO
0001:000a7711* _X509_CRL_INFO_new
0001:000a7725* _X509_CRL_INFO_free
0001:000a7740* _d2i_X509_CRL
0001:000a7769* _i2d_X509_CRL
0001:000a778b* _X509_CRL_new
0001:000a779f  _X509_CRL_free
0001:000a77ba* _X509_CRL_dup
0001:000a77ff* _X509_CRL_add0_revoked
0001:000a7893  _X509_CRL_verify
0001:000a78c7* _X509_CRL_get0_by_serial
0001:000a790a  _X509_CRL_get0_by_cert
0001:000a7bae* _X509_CRL_set_default_method
0001:000a7bcd* _X509_CRL_METHOD_new
0001:000a7c31* _X509_CRL_METHOD_free
0001:000a7c53* _X509_CRL_set_meth_data
0001:000a7c61* _X509_CRL_get_meth_data
Module: U:\extras\lib\libcrypto.lib(ecp_smpl.obj)
0001:000a7c70* _EC_GFp_simple_method
0001:000a7c7a  _ec_GFp_simple_group_init
0001:000a7cc0  _ec_GFp_simple_group_finish
0001:000a7cf4  _ec_GFp_simple_group_clear_finish
0001:000a7d28  _ec_GFp_simple_group_copy
0001:000a7dc0  _ec_GFp_simple_group_set_curve
0001:000a8028  _ec_GFp_simple_group_get_curve
0001:000a8185  _ec_GFp_simple_group_get_degree
0001:000a819b  _ec_GFp_simple_group_check_discriminant
0001:000a8476  _ec_GFp_simple_point_init
0001:000a84b7  _ec_GFp_simple_point_finish
0001:000a84e9  _ec_GFp_simple_point_clear_finish
0001:000a8525  _ec_GFp_simple_point_copy
0001:000a85a7  _ec_GFp_simple_point_set_to_infinity
0001:000a85d4  _ec_GFp_simple_set_Jprojective_coordinates_GFp
0001:000a8827  _ec_GFp_simple_get_Jprojective_coordinates_GFp
0001:000a89a8  _ec_GFp_simple_point_set_affine_coordinates
0001:000a8a1f  _ec_GFp_simple_point_get_affine_coordinates
0001:000a8e4d  _ec_GFp_simple_set_compressed_coordinates
0001:000a9464  _ec_GFp_simple_point2oct
0001:000a9866  _ec_GFp_simple_oct2point
0001:000a9ca4  _ec_GFp_simple_add
0001:000aa4a5  _ec_GFp_simple_dbl
0001:000aab4d  _ec_GFp_simple_invert
0001:000aab9e  _ec_GFp_simple_is_at_infinity
0001:000aabb1  _ec_GFp_simple_is_on_curve
0001:000aaff9  _ec_GFp_simple_cmp
0001:000ab3a3  _ec_GFp_simple_make_affine
0001:000ab4f5  _ec_GFp_simple_points_make_affine
0001:000abbee* _ec_GFp_simple_field_mul
0001:000abc20* _ec_GFp_simple_field_sqr
Module: U:\extras\lib\libcrypto.lib(bn_nist.obj)
0001:000ac194  _BN_get0_nist_prime_192
0001:000ac19e  _BN_get0_nist_prime_224
0001:000ac1a8  _BN_get0_nist_prime_256
0001:000ac1b2  _BN_get0_nist_prime_384
0001:000ac1bc  _BN_get0_nist_prime_521
0001:000ac25b  _BN_nist_mod_192
0001:000ac56a  _BN_nist_mod_224
0001:000ac994  _BN_nist_mod_256
0001:000acf2c  _BN_nist_mod_384
0001:000ad5ca  _BN_nist_mod_521
Module: U:\extras\lib\libcrypto.lib(bn_gf2m.obj)
0001:000adbd1  _BN_GF2m_add
0001:000add16  _BN_GF2m_mod_arr
0001:000ae180* _BN_GF2m_mod
0001:000af5e4  _BN_GF2m_poly2arr
0001:000ae257  _BN_GF2m_mod_mul_arr
0001:000ae5c3  _BN_GF2m_mod_sqr_arr
0001:000ae4da* _BN_GF2m_mod_mul
0001:000ae807* _BN_GF2m_mod_sqr
0001:000ae8e5* _BN_GF2m_mod_inv
0001:000aeb36* _BN_GF2m_mod_inv_arr
0001:000af6a0* _BN_GF2m_arr2poly
0001:000aebb1  _BN_GF2m_mod_div
0001:000aec53* _BN_GF2m_mod_div_arr
0001:000aecd5* _BN_GF2m_mod_exp_arr
0001:000aee40* _BN_GF2m_mod_exp
0001:000aef29  _BN_GF2m_mod_sqrt_arr
0001:000aefd1* _BN_GF2m_mod_sqrt
0001:000af0af  _BN_GF2m_mod_solve_quad_arr
0001:000af506* _BN_GF2m_mod_solve_quad
Module: U:\extras\lib\libcrypto.lib(ec2_mult.obj)
0001:000b0330  _ec_GF2m_simple_mul
0001:000b05f5  _ec_GF2m_precompute_mult
0001:000b060f  _ec_GF2m_have_precompute_mult
Module: U:\extras\lib\libcrypto.lib(v3_pcia.obj)
0001:000b0690* _PROXY_POLICY_it
0001:000b06ac* _d2i_PROXY_POLICY
0001:000b06d5* _i2d_PROXY_POLICY
0001:000b06f7* _PROXY_POLICY_new
0001:000b070b* _PROXY_POLICY_free
0001:000b07a0  _PROXY_CERT_INFO_EXTENSION_it
0001:000b07bc* _d2i_PROXY_CERT_INFO_EXTENSION
0001:000b07e5* _i2d_PROXY_CERT_INFO_EXTENSION
0001:000b0807  _PROXY_CERT_INFO_EXTENSION_new
0001:000b081b  _PROXY_CERT_INFO_EXTENSION_free
Module: U:\extras\lib\libcrypto.lib(a_strex.obj)
0001:000b16eb  _X509_NAME_print_ex
0001:000b173c* _X509_NAME_print_ex_fp
0001:000b17c1  _ASN1_STRING_print_ex
0001:000b17ea* _ASN1_STRING_print_ex_fp
0001:000b1813  _ASN1_STRING_to_UTF8
Module: U:\extras\lib\libcrypto.lib(asn1_gen.obj)
0001:000b18e0* _ASN1_generate_nconf
0001:000b1932  _ASN1_generate_v3
Module: U:\extras\lib\libcrypto.lib(a_verify.obj)
0001:000b32db* _ASN1_verify
0001:000b34a1  _ASN1_item_verify
Module: U:\extras\lib\libcrypto.lib(x_spki.obj)
0001:000b3770  _NETSCAPE_SPKAC_it
0001:000b378c* _d2i_NETSCAPE_SPKAC
0001:000b37b5* _i2d_NETSCAPE_SPKAC
0001:000b37d7* _NETSCAPE_SPKAC_new
0001:000b37eb* _NETSCAPE_SPKAC_free
0001:000b3870* _NETSCAPE_SPKI_it
0001:000b388c* _d2i_NETSCAPE_SPKI
0001:000b38b5* _i2d_NETSCAPE_SPKI
0001:000b38d7* _NETSCAPE_SPKI_new
0001:000b38eb* _NETSCAPE_SPKI_free
Module: U:\extras\lib\libcrypto.lib(a_sign.obj)
0001:000b3919* _ASN1_sign
0001:000b3c84  _ASN1_item_sign
Module: U:\extras\lib\libcrypto.lib(pk7_asn1.obj)
0001:000b43d0* _PKCS7_SIGNED_it
0001:000b4790* _PKCS7_ENVELOPE_it
0001:000b4b30* _PKCS7_SIGN_ENVELOPE_it
0001:000b4d10* _PKCS7_DIGEST_it
0001:000b4c10* _PKCS7_ENCRYPT_it
0001:000b4230  _PKCS7_it
0001:000b424c* _d2i_PKCS7
0001:000b4275* _i2d_PKCS7
0001:000b4297  _PKCS7_new
0001:000b42ab  _PKCS7_free
0001:000b42c6* _i2d_PKCS7_NDEF
0001:000b42e8* _PKCS7_dup
0001:000b45a0* _PKCS7_SIGNER_INFO_it
0001:000b43ec* _d2i_PKCS7_SIGNED
0001:000b4415* _i2d_PKCS7_SIGNED
0001:000b4437  _PKCS7_SIGNED_new
0001:000b444b  _PKCS7_SIGNED_free
0001:000b4690  _PKCS7_ISSUER_AND_SERIAL_it
0001:000b45bc* _d2i_PKCS7_SIGNER_INFO
0001:000b45e5* _i2d_PKCS7_SIGNER_INFO
0001:000b4607  _PKCS7_SIGNER_INFO_new
0001:000b461b  _PKCS7_SIGNER_INFO_free
0001:000b46ac* _d2i_PKCS7_ISSUER_AND_SERIAL
0001:000b46d5* _i2d_PKCS7_ISSUER_AND_SERIAL
0001:000b46f7* _PKCS7_ISSUER_AND_SERIAL_new
0001:000b470b* _PKCS7_ISSUER_AND_SERIAL_free
0001:000b48f0* _PKCS7_RECIP_INFO_it
0001:000b49f0* _PKCS7_ENC_CONTENT_it
0001:000b47ac* _d2i_PKCS7_ENVELOPE
0001:000b47d5* _i2d_PKCS7_ENVELOPE
0001:000b47f7  _PKCS7_ENVELOPE_new
0001:000b480b* _PKCS7_ENVELOPE_free
0001:000b490c* _d2i_PKCS7_RECIP_INFO
0001:000b4935* _i2d_PKCS7_RECIP_INFO
0001:000b4957  _PKCS7_RECIP_INFO_new
0001:000b496b  _PKCS7_RECIP_INFO_free
0001:000b4a0c* _d2i_PKCS7_ENC_CONTENT
0001:000b4a35* _i2d_PKCS7_ENC_CONTENT
0001:000b4a57* _PKCS7_ENC_CONTENT_new
0001:000b4a6b* _PKCS7_ENC_CONTENT_free
0001:000b4b4c* _d2i_PKCS7_SIGN_ENVELOPE
0001:000b4b75* _i2d_PKCS7_SIGN_ENVELOPE
0001:000b4b97  _PKCS7_SIGN_ENVELOPE_new
0001:000b4bab* _PKCS7_SIGN_ENVELOPE_free
0001:000b4c2c* _d2i_PKCS7_ENCRYPT
0001:000b4c55* _i2d_PKCS7_ENCRYPT
0001:000b4c77  _PKCS7_ENCRYPT_new
0001:000b4c8b* _PKCS7_ENCRYPT_free
0001:000b4d2c* _d2i_PKCS7_DIGEST
0001:000b4d55* _i2d_PKCS7_DIGEST
0001:000b4d77  _PKCS7_DIGEST_new
0001:000b4d8b* _PKCS7_DIGEST_free
0001:000b4df0  _PKCS7_ATTR_SIGN_it
0001:000b4e40  _PKCS7_ATTR_VERIFY_it
0001:000b4e5c* _PKCS7_print_ctx
Module: U:\extras\lib\libcrypto.lib(a_digest.obj)
0001:000b4e9b* _ASN1_digest
0001:000b4f67  _ASN1_item_digest
Module: U:\extras\lib\libcrypto.lib(evp_pkey.obj)
0001:000b4ff1  _EVP_PKCS82PKEY
0001:000b519d  _EVP_PKEY2PKCS8
0001:000b51b8* _EVP_PKEY2PKCS8_broken
0001:000b5323* _PKCS8_set_broken
0001:000b5392* _EVP_PKEY_get_attr_count
0001:000b53a8* _EVP_PKEY_get_attr_by_NID
0001:000b53cc* _EVP_PKEY_get_attr_by_OBJ
0001:000b53f0* _EVP_PKEY_get_attr
0001:000b540d* _EVP_PKEY_delete_attr
0001:000b542a* _EVP_PKEY_add1_attr
0001:000b5457* _EVP_PKEY_add1_attr_by_OBJ
0001:000b5499* _EVP_PKEY_add1_attr_by_NID
0001:000b54db* _EVP_PKEY_add1_attr_by_txt
Module: U:\extras\lib\libcrypto.lib(i2d_pr.obj)
0001:000b5529  _i2d_PrivateKey
Module: U:\extras\lib\libcrypto.lib(d2i_pr.obj)
0001:000b55e9* _d2i_PrivateKey
0001:000b57b1  _d2i_AutoPrivateKey
Module: U:\extras\lib\libcrypto.lib(t_x509.obj)
0001:000b5900* _X509_print_fp
0001:000b5933* _X509_print_ex_fp
0001:000b5b71* _X509_print_ex
0001:000b59d7* _X509_print
0001:000b667d* _ASN1_TIME_print
0001:000b645a* _X509_signature_print
0001:000b624c* _X509_ocspid_print
0001:000b657d  _ASN1_STRING_print
0001:000b6ab1  _ASN1_UTCTIME_print
0001:000b6737  _ASN1_GENERALIZEDTIME_print
0001:000b6d49  _X509_NAME_print
Module: U:\extras\lib\libcrypto.lib(v3_akeya.obj)
0001:000b6f30  _AUTHORITY_KEYID_it
0001:000b6f4c* _d2i_AUTHORITY_KEYID
0001:000b6f75* _i2d_AUTHORITY_KEYID
0001:000b6f97  _AUTHORITY_KEYID_new
0001:000b6fab  _AUTHORITY_KEYID_free
Module: U:\extras\lib\libcrypto.lib(ocsp_asn.obj)
0001:000b7050* _OCSP_SIGNATURE_it
0001:000b706c* _d2i_OCSP_SIGNATURE
0001:000b7095* _i2d_OCSP_SIGNATURE
0001:000b70b7* _OCSP_SIGNATURE_new
0001:000b70cb* _OCSP_SIGNATURE_free
0001:000b7180* _OCSP_CERTID_it
0001:000b719c* _d2i_OCSP_CERTID
0001:000b71c5* _i2d_OCSP_CERTID
0001:000b71e7* _OCSP_CERTID_new
0001:000b71fb* _OCSP_CERTID_free
0001:000b7280* _OCSP_ONEREQ_it
0001:000b729c* _d2i_OCSP_ONEREQ
0001:000b72c5* _i2d_OCSP_ONEREQ
0001:000b72e7* _OCSP_ONEREQ_new
0001:000b72fb* _OCSP_ONEREQ_free
0001:000b73b0* _OCSP_REQINFO_it
0001:000b73cc* _d2i_OCSP_REQINFO
0001:000b73f5* _i2d_OCSP_REQINFO
0001:000b7417* _OCSP_REQINFO_new
0001:000b742b* _OCSP_REQINFO_free
0001:000b74b0* _OCSP_REQUEST_it
0001:000b74cc* _d2i_OCSP_REQUEST
0001:000b74f5* _i2d_OCSP_REQUEST
0001:000b7517* _OCSP_REQUEST_new
0001:000b752b* _OCSP_REQUEST_free
0001:000b75a0* _OCSP_RESPBYTES_it
0001:000b75bc* _d2i_OCSP_RESPBYTES
0001:000b75e5* _i2d_OCSP_RESPBYTES
0001:000b7607* _OCSP_RESPBYTES_new
0001:000b761b* _OCSP_RESPBYTES_free
0001:000b76a0* _OCSP_RESPONSE_it
0001:000b76bc* _d2i_OCSP_RESPONSE
0001:000b76e5* _i2d_OCSP_RESPONSE
0001:000b7707* _OCSP_RESPONSE_new
0001:000b771b* _OCSP_RESPONSE_free
0001:000b7790* _OCSP_RESPID_it
0001:000b77ac* _d2i_OCSP_RESPID
0001:000b77d5* _i2d_OCSP_RESPID
0001:000b77f7* _OCSP_RESPID_new
0001:000b780b* _OCSP_RESPID_free
0001:000b7890* _OCSP_REVOKEDINFO_it
0001:000b78ac* _d2i_OCSP_REVOKEDINFO
0001:000b78d5* _i2d_OCSP_REVOKEDINFO
0001:000b78f7* _OCSP_REVOKEDINFO_new
0001:000b790b* _OCSP_REVOKEDINFO_free
0001:000b79a0* _OCSP_CERTSTATUS_it
0001:000b79bc* _d2i_OCSP_CERTSTATUS
0001:000b79e5* _i2d_OCSP_CERTSTATUS
0001:000b7a07* _OCSP_CERTSTATUS_new
0001:000b7a1b* _OCSP_CERTSTATUS_free
0001:000b7af0* _OCSP_SINGLERESP_it
0001:000b7b0c* _d2i_OCSP_SINGLERESP
0001:000b7b35* _i2d_OCSP_SINGLERESP
0001:000b7b57* _OCSP_SINGLERESP_new
0001:000b7b6b* _OCSP_SINGLERESP_free
0001:000b7c40* _OCSP_RESPDATA_it
0001:000b7c5c* _d2i_OCSP_RESPDATA
0001:000b7c85* _i2d_OCSP_RESPDATA
0001:000b7ca7* _OCSP_RESPDATA_new
0001:000b7cbb* _OCSP_RESPDATA_free
0001:000b7d50* _OCSP_BASICRESP_it
0001:000b7d6c* _d2i_OCSP_BASICRESP
0001:000b7d95* _i2d_OCSP_BASICRESP
0001:000b7db7* _OCSP_BASICRESP_new
0001:000b7dcb* _OCSP_BASICRESP_free
0001:000b7e50  _OCSP_CRLID_it
0001:000b7e6c* _d2i_OCSP_CRLID
0001:000b7e95* _i2d_OCSP_CRLID
0001:000b7eb7* _OCSP_CRLID_new
0001:000b7ecb* _OCSP_CRLID_free
0001:000b7f40  _OCSP_SERVICELOC_it
0001:000b7f5c* _d2i_OCSP_SERVICELOC
0001:000b7f85* _i2d_OCSP_SERVICELOC
0001:000b7fa7* _OCSP_SERVICELOC_new
0001:000b7fbb* _OCSP_SERVICELOC_free
Module: U:\extras\lib\libcrypto.lib(f_int.obj)
0001:000b7fe8  _i2a_ASN1_INTEGER
0001:000b8156* _a2i_ASN1_INTEGER
Module: U:\extras\lib\libcrypto.lib(f_string.obj)
0001:000b8565  _i2a_ASN1_STRING
0001:000b869c* _a2i_ASN1_STRING
Module: U:\extras\lib\libcrypto.lib(a_mbstr.obj)
0001:000b8a80  _ASN1_mbstring_copy
0001:000b8adf  _ASN1_mbstring_ncopy
Module: U:\extras\lib\libcrypto.lib(conf_def.obj)
0001:000b94a0* _CONF_def_version
0001:000b94e2  _NCONF_default
0001:000b94ec* _NCONF_WIN32
Module: U:\extras\lib\libcrypto.lib(conf_api.obj)
0001:000baa9f  __CONF_get_section
0001:000baae2  __CONF_get_section_values
0001:000bab12  __CONF_add_string
0001:000babb9  __CONF_get_string
0001:000bad93  __CONF_new_data
0001:000bade4  __CONF_free_data
0001:000baf2e  __CONF_new_section
Module: U:\extras\lib\libcrypto.lib(dso_openssl.obj)
0001:000bb070  _DSO_METHOD_openssl
Module: U:\extras\lib\libcrypto.lib(cms_asn1.obj)
0001:000bb0f0  _CMS_IssuerAndSerialNumber_it
0001:000bb180* _CMS_OtherCertificateFormat_it
0001:000bb270  _CMS_CertificateChoices_it
0001:000bb300* _CMS_SignerIdentifier_it
0001:000bb390* _CMS_EncapsulatedContentInfo_it
0001:000bb510  _CMS_SignerInfo_it
0001:000bb5a0* _CMS_OtherRevocationInfoFormat_it
0001:000bb620  _CMS_RevocationInfoChoice_it
0001:000bb710  _CMS_SignedData_it
0001:000bb770* _CMS_OriginatorInfo_it
0001:000bb830* _CMS_EncryptedContentInfo_it
0001:000bb8f0  _CMS_KeyTransRecipientInfo_it
0001:000bb960  _CMS_OtherKeyAttribute_it
0001:000bba00* _CMS_RecipientKeyIdentifier_it
0001:000bba80* _CMS_KeyAgreeRecipientIdentifier_it
0001:000bbaf0* _CMS_RecipientEncryptedKey_it
0001:000bbb60* _CMS_OriginatorPublicKey_it
0001:000bbbf0* _CMS_OriginatorIdentifierOrKey_it
0001:000bbcc0* _CMS_KeyAgreeRecipientInfo_it
0001:000bbd40* _CMS_KEKIdentifier_it
0001:000bbde0  _CMS_KEKRecipientInfo_it
0001:000bbe90* _CMS_PasswordRecipientInfo_it
0001:000bbf00* _CMS_OtherRecipientInfo_it
0001:000bc090  _CMS_RecipientInfo_it
0001:000bc170  _CMS_EnvelopedData_it
0001:000bc210  _CMS_DigestedData_it
0001:000bc280  _CMS_EncryptedData_it
0001:000bc3a0* _CMS_AuthenticatedData_it
0001:000bc430* _CMS_CompressedData_it
0001:000bc6c0  _CMS_ContentInfo_it
0001:000bc720  _CMS_Attributes_Sign_it
0001:000bc770  _CMS_Attributes_Verify_it
0001:000bc7f0* _CMS_ReceiptsFrom_it
0001:000bc890* _CMS_ReceiptRequest_it
0001:000bc930* _CMS_Receipt_it
Module: U:\extras\lib\libcrypto.lib(cms_att.obj)
0001:000bc950  _CMS_signed_get_attr_count
0001:000bc966  _CMS_signed_get_attr_by_NID
0001:000bc98a* _CMS_signed_get_attr_by_OBJ
0001:000bc9ae* _CMS_signed_get_attr
0001:000bc9cb* _CMS_signed_delete_attr
0001:000bc9e8* _CMS_signed_add1_attr
0001:000bca15* _CMS_signed_add1_attr_by_OBJ
0001:000bca57  _CMS_signed_add1_attr_by_NID
0001:000bca99* _CMS_signed_add1_attr_by_txt
0001:000bcadb  _CMS_signed_get0_data_by_OBJ
0001:000bcb06* _CMS_unsigned_get_attr_count
0001:000bcb1c* _CMS_unsigned_get_attr_by_NID
0001:000bcb40* _CMS_unsigned_get_attr_by_OBJ
0001:000bcb64* _CMS_unsigned_get_attr
0001:000bcb81* _CMS_unsigned_delete_attr
0001:000bcb9e* _CMS_unsigned_add1_attr
0001:000bcbcb* _CMS_unsigned_add1_attr_by_OBJ
0001:000bcc0d* _CMS_unsigned_add1_attr_by_NID
0001:000bcc4f* _CMS_unsigned_add1_attr_by_txt
0001:000bcc91* _CMS_unsigned_get0_data_by_OBJ
Module: U:\extras\lib\libcrypto.lib(cms_lib.obj)
0001:000bccc0  _d2i_CMS_ContentInfo
0001:000bcce9  _i2d_CMS_ContentInfo
0001:000bcd0b  _CMS_ContentInfo_new
0001:000bcd1f  _CMS_ContentInfo_free
0001:000bcd3a* _CMS_ContentInfo_print_ctx
0001:000bcd6a* _CMS_get0_type
0001:000bcd74* _priv_cms_Data_create
0001:000bd3a3* _CMS_set_detached
0001:000bcdb1* _cms_content_bio
0001:000bd138  _CMS_get0_content
0001:000bce36  _CMS_dataInit
0001:000bcf79  _CMS_dataFinal
0001:000bd2de  _CMS_get0_eContentType
0001:000bd306* _CMS_set1_eContentType
0001:000bd36b* _CMS_is_detached
0001:000bd45c  _cms_DigestAlgorithm_set
0001:000bd4b2  _cms_DigestAlgorithm_init_bio
0001:000bd5ba  _cms_DigestAlgorithm_find_ctx
0001:000bd727* _CMS_add0_CertificateChoices
0001:000bd7c0* _CMS_add0_cert
0001:000bd8b6  _CMS_add1_cert
0001:000bd975* _CMS_add0_RevocationInfoChoice
0001:000bda0e* _CMS_add0_crl
0001:000bda48* _CMS_add1_crl
0001:000bda9c* _CMS_get1_certs
0001:000bdb98* _CMS_get1_crls
Module: U:\extras\lib\libcrypto.lib(x509_vfy.obj)
0001:000bdca0* _X509_version
0001:000bdcdc  _X509_verify_cert
0001:000c0a25* _X509_get_pubkey_parameters
0001:000c065b* _X509_cmp_time
0001:000c0fa2  _X509_STORE_CTX_init
0001:000c1523* _X509_STORE_CTX_set0_param
0001:000c1391  _X509_STORE_CTX_cleanup
0001:000c0640* _X509_cmp_current_time
0001:000c094c* _X509_time_adj
0001:000c092a  _X509_gmtime_adj
0001:000c0975* _X509_time_adj_ex
0001:000c0b9d* _X509_STORE_CTX_get_ex_new_index
0001:000c0bd4* _X509_STORE_CTX_set_ex_data
0001:000c0bfb* _X509_STORE_CTX_get_ex_data
0001:000c0c1b* _X509_STORE_CTX_get_error
0001:000c0c26* _X509_STORE_CTX_set_error
0001:000c0c34* _X509_STORE_CTX_get_error_depth
0001:000c0c3f* _X509_STORE_CTX_get_current_cert
0001:000c0c4a* _X509_STORE_CTX_get_chain
0001:000c0c55* _X509_STORE_CTX_get1_chain
0001:000c0ce7* _X509_STORE_CTX_get0_current_issuer
0001:000c0cf2* _X509_STORE_CTX_get0_current_crl
0001:000c0cfd* _X509_STORE_CTX_get0_parent_ctx
0001:000c0d08* _X509_STORE_CTX_set_cert
0001:000c0d16* _X509_STORE_CTX_set_chain
0001:000c0d24* _X509_STORE_CTX_set0_crls
0001:000c0d32  _X509_STORE_CTX_set_purpose
0001:000c0d86* _X509_STORE_CTX_purpose_inherit
0001:000c0d5c* _X509_STORE_CTX_set_trust
0001:000c0efe* _X509_STORE_CTX_new
0001:000c0f7c* _X509_STORE_CTX_free
0001:000c1379* _X509_STORE_CTX_trusted_stack
0001:000c1465* _X509_STORE_CTX_set_depth
0001:000c1482* _X509_STORE_CTX_set_flags
0001:000c149f* _X509_STORE_CTX_set_time
0001:000c14bc* _X509_STORE_CTX_set_verify_cb
0001:000c14ca* _X509_STORE_CTX_get0_policy_tree
0001:000c14d5* _X509_STORE_CTX_get_explicit_policy
0001:000c14e0* _X509_STORE_CTX_set_default
0001:000c1518* _X509_STORE_CTX_get0_param
Module: U:\extras\lib\libcrypto.lib(a_time.obj)
0001:000c1560  _ASN1_TIME_it
0001:000c157c* _d2i_ASN1_TIME
0001:000c15a5* _i2d_ASN1_TIME
0001:000c15c7* _ASN1_TIME_new
0001:000c15db  _ASN1_TIME_free
0001:000c15f6* _ASN1_TIME_set
0001:000c1629  _ASN1_TIME_adj
0001:000c170c  _ASN1_TIME_check
0001:000c174f* _ASN1_TIME_to_generalizedtime
0001:000c1890* _ASN1_TIME_set_string
Module: U:\extras\lib\libcrypto.lib(p_sign.obj)
0001:000c1919  _EVP_SignFinal
Module: U:\extras\lib\libcrypto.lib(m_sigver.obj)
0001:000c1d5e  _EVP_DigestSignInit
0001:000c1d95  _EVP_DigestVerifyInit
0001:000c1dcc  _EVP_DigestSignFinal
0001:000c1f66  _EVP_DigestVerifyFinal
Module: U:\extras\lib\libcrypto.lib(p_verify.obj)
0001:000c206b  _EVP_VerifyFinal
Module: U:\extras\lib\libcrypto.lib(cms_enc.obj)
0001:000c229a  _cms_EncryptedContent_init_bio
0001:000c274d  _cms_EncryptedContent_init
0001:000c27d9* _CMS_EncryptedData_set1_key
0001:000c290d  _cms_EncryptedData_init_bio
Module: U:\extras\lib\libcrypto.lib(pmeth_fn.obj)
0001:000c295b  _EVP_PKEY_sign_init
0001:000c29f4  _EVP_PKEY_sign
0001:000c2b2c  _EVP_PKEY_verify_init
0001:000c2bc5  _EVP_PKEY_verify
0001:000c2c85* _EVP_PKEY_verify_recover_init
0001:000c2d1e* _EVP_PKEY_verify_recover
0001:000c2e56  _EVP_PKEY_encrypt_init
0001:000c2eef  _EVP_PKEY_encrypt
0001:000c3029  _EVP_PKEY_decrypt_init
0001:000c30c2  _EVP_PKEY_decrypt
0001:000c31fc* _EVP_PKEY_derive_init
0001:000c3295* _EVP_PKEY_derive_set_peer
0001:000c352f* _EVP_PKEY_derive
Module: U:\extras\lib\libcrypto.lib(aes_core.obj)
0001:000c5788  _AES_set_encrypt_key
0001:000c5e25  _AES_set_decrypt_key
0001:000c61e8  _AES_encrypt
0001:000c6847  _AES_decrypt
Module: U:\extras\lib\libcrypto.lib(aes_wrap.obj)
0001:000c6ea8  _AES_wrap_key
0001:000c7038  _AES_unwrap_key
Module: U:\extras\lib\libcrypto.lib(x_val.obj)
0001:000c7260  _X509_VAL_it
0001:000c727c* _d2i_X509_VAL
0001:000c72a5* _i2d_X509_VAL
0001:000c72c7* _X509_VAL_new
0001:000c72db* _X509_VAL_free
Module: U:\extras\lib\libcrypto.lib(x_x509a.obj)
0001:000c73a0* _X509_CERT_AUX_it
0001:000c73bc  _d2i_X509_CERT_AUX
0001:000c73e5  _i2d_X509_CERT_AUX
0001:000c7407* _X509_CERT_AUX_new
0001:000c741b  _X509_CERT_AUX_free
0001:000c7477* _X509_alias_set1
0001:000c752e* _X509_keyid_set1
0001:000c75e5* _X509_alias_get0
0001:000c762a* _X509_keyid_get0
0001:000c766f* _X509_add1_trust_object
0001:000c76e6* _X509_add1_reject_object
0001:000c7761* _X509_trust_clear
0001:000c77a4* _X509_reject_clear
0001:000c7840* _X509_CERT_PAIR_it
0001:000c785c* _d2i_X509_CERT_PAIR
0001:000c7885* _i2d_X509_CERT_PAIR
0001:000c78a7* _X509_CERT_PAIR_new
0001:000c78bb* _X509_CERT_PAIR_free
Module: U:\extras\lib\libcrypto.lib(pcy_cache.obj)
0001:000c7d00  _policy_cache_free
0001:000c7d53  _policy_cache_set
0001:000c7dbe  _policy_cache_find_data
Module: U:\extras\lib\libcrypto.lib(p12_p8e.obj)
0001:000c7e7a  _PKCS8_encrypt
Module: U:\extras\lib\libcrypto.lib(p12_decr.obj)
0001:000c800b* _PKCS12_pbe_crypt
0001:000c81bd  _PKCS12_item_decrypt_d2i
0001:000c82c5  _PKCS12_item_i2d_encrypt
Module: U:\extras\lib\libcrypto.lib(p12_p8d.obj)
0001:000c8420  _PKCS8_decrypt
Module: U:\extras\lib\libcrypto.lib(bn_sqrt.obj)
0001:000c846a  _BN_mod_sqrt
Module: U:\extras\lib\libcrypto.lib(bn_kron.obj)
0001:000c8fc0  _BN_kronecker
Module: U:\extras\lib\libcrypto.lib(a_utf8.obj)
0001:000c9340  _UTF8_getc
0001:000c97f0  _UTF8_putc
Module: U:\extras\lib\libcrypto.lib(asn1_par.obj)
0001:000ca85e  _ASN1_tag2str
0001:000c9c4e* _ASN1_parse
0001:000c9c8e  _ASN1_parse_dump
Module: U:\extras\lib\libcrypto.lib(pk7_doit.obj)
0001:000cb063  _PKCS7_dataInit
0001:000cb656* _PKCS7_dataDecode
0001:000ccde5  _PKCS7_get_signed_attribute
0001:000cc532* _PKCS7_SIGNER_INFO_sign
0001:000cbf88  _PKCS7_dataFinal
0001:000cc7a9* _PKCS7_dataVerify
0001:000cc971* _PKCS7_signatureVerify
0001:000cced4* _PKCS7_digest_from_attributes
0001:000ccd4d* _PKCS7_get_issuer_and_serial
0001:000cce02* _PKCS7_get_attribute
0001:000ccf05* _PKCS7_set_signed_attributes
0001:000ccfb1* _PKCS7_set_attributes
0001:000cd05d  _PKCS7_add_signed_attribute
0001:000cd088* _PKCS7_add_attribute
Module: U:\extras\lib\libcrypto.lib(tasn_prn.obj)
0001:000cd21b* _ASN1_PCTX_new
0001:000cd2af* _ASN1_PCTX_free
0001:000cd2c2* _ASN1_PCTX_get_flags
0001:000cd2cc* _ASN1_PCTX_set_flags
0001:000cd2d9* _ASN1_PCTX_get_nm_flags
0001:000cd2e4* _ASN1_PCTX_set_nm_flags
0001:000cd2f2* _ASN1_PCTX_get_cert_flags
0001:000cd2fd* _ASN1_PCTX_set_cert_flags
0001:000cd30b* _ASN1_PCTX_get_oid_flags
0001:000cd316* _ASN1_PCTX_set_oid_flags
0001:000cd324* _ASN1_PCTX_get_str_flags
0001:000cd32f* _ASN1_PCTX_set_str_flags
0001:000cd33d  _ASN1_item_print
0001:000cd98f* _asn1_template_print_ctx
0002:000013f0* _default_pctx
Module: U:\extras\lib\libcrypto.lib(err_prn.obj)
0001:000ce332  _ERR_print_errors_cb
0001:000ce4a5* _ERR_print_errors_fp
0001:000ce4e1  _ERR_print_errors
Module: U:\extras\lib\libcrypto.lib(v3_prn.obj)
0001:000ce519* _X509V3_EXT_val_prn
0001:000ce68a* _X509V3_EXT_print
0001:000ce8fd  _X509V3_extensions_print
0001:000cebd6* _X509V3_EXT_print_fp
Module: U:\extras\lib\libcrypto.lib(t_x509a.obj)
0001:000cecbf  _X509_CERT_AUX_print
Module: U:\extras\lib\libcrypto.lib(dso_null.obj)
0001:000cefdb  _DSO_METHOD_null
Module: U:\extras\lib\libcrypto.lib(cms_io.obj)
0001:000ceff9  _CMS_stream
0001:000cf0a6* _d2i_CMS_bio
0001:000cf0c8* _i2d_CMS_bio
0001:000cf0ee* _PEM_read_bio_CMS
0001:000cf127* _PEM_read_CMS
0001:000cf160* _PEM_write_bio_CMS
0001:000cf1b3* _PEM_write_CMS
0001:000cf206* _BIO_new_CMS
0001:000cf228* _i2d_CMS_bio_stream
0001:000cf258* _PEM_write_bio_CMS_stream
0001:000cf290* _SMIME_write_CMS
0001:000cf316* _SMIME_read_CMS
Module: U:\extras\lib\libcrypto.lib(bss_null.obj)
0001:000cf345  _BIO_s_null
Module: U:\extras\lib\libcrypto.lib(bss_mem.obj)
0001:000cf44e  _BIO_s_mem
0001:000cf462  _BIO_new_mem_buf
Module: U:\extras\lib\libcrypto.lib(cms_dd.obj)
0001:000cfa90* _cms_DigestedData_create
0001:000cfb2f  _cms_DigestedData_init_bio
0001:000cfb57  _cms_DigestedData_do_final
Module: U:\extras\lib\libcrypto.lib(bio_md.obj)
0001:000cfcbf  _BIO_f_md
Module: U:\extras\lib\libcrypto.lib(x509_trs.obj)
0001:000d01cc* _X509_TRUST_set_default
0001:000d01e7  _X509_check_trust
0001:000d02c7  _X509_TRUST_get_by_id
0001:000d0280* _X509_TRUST_get0
0001:000d0258* _X509_TRUST_get_count
0001:000d032c  _X509_TRUST_set
0001:000d0384* _X509_TRUST_add
0001:000d05c3* _X509_TRUST_cleanup
0001:000d0616* _X509_TRUST_get_flags
0001:000d0621* _X509_TRUST_get0_name
0001:000d062c* _X509_TRUST_get_trust
Module: U:\extras\lib\libcrypto.lib(pcy_tree.obj)
0001:000d1552  _X509_policy_tree_free
0001:000d1637  _X509_policy_check
Module: U:\extras\lib\libcrypto.lib(a_utctm.obj)
0001:000d1800  _ASN1_UTCTIME_check
0001:000d1a48* _ASN1_UTCTIME_set_string
0001:000d1aba* _ASN1_UTCTIME_set
0001:000d1b08  _ASN1_UTCTIME_adj
0001:000d1cdb* _ASN1_UTCTIME_cmp_time_t
Module: U:\extras\lib\libcrypto.lib(a_gentm.obj)
0001:000d2120  _ASN1_GENERALIZEDTIME_check
0001:000d23c0* _ASN1_GENERALIZEDTIME_set_string
0001:000d2432* _ASN1_GENERALIZEDTIME_set
0001:000d2480  _ASN1_GENERALIZEDTIME_adj
Module: U:\extras\lib\libcrypto.lib(x509_vpm.obj)
0001:000d2712  _X509_VERIFY_PARAM_new
0001:000d2762  _X509_VERIFY_PARAM_free
0001:000d2780  _X509_VERIFY_PARAM_inherit
0001:000d2aca* _X509_VERIFY_PARAM_set1_policies
0001:000d2928  _X509_VERIFY_PARAM_set1
0001:000d296b* _X509_VERIFY_PARAM_set1_name
0001:000d29ae  _X509_VERIFY_PARAM_set_flags
0001:000d29e6* _X509_VERIFY_PARAM_clear_flags
0001:000d2a03* _X509_VERIFY_PARAM_get_flags
0001:000d2a0e  _X509_VERIFY_PARAM_set_purpose
0001:000d2a2b  _X509_VERIFY_PARAM_set_trust
0001:000d2a48  _X509_VERIFY_PARAM_set_depth
0001:000d2a56  _X509_VERIFY_PARAM_set_time
0001:000d2a75* _X509_VERIFY_PARAM_add0_policy
0001:000d2bcb* _X509_VERIFY_PARAM_get_depth
0001:000d2d47* _X509_VERIFY_PARAM_add0_table
0001:000d2df1  _X509_VERIFY_PARAM_lookup
0001:000d2e56* _X509_VERIFY_PARAM_table_cleanup
Module: U:\extras\lib\libcrypto.lib(x509_lu.obj)
0001:000d2e9a* _X509_LOOKUP_new
0001:000d2f2f* _X509_LOOKUP_free
0001:000d2f73* _X509_LOOKUP_init
0001:000d2fb1* _X509_LOOKUP_shutdown
0001:000d2fef* _X509_LOOKUP_ctrl
0001:000d3049* _X509_LOOKUP_by_subject
0001:000d30a6* _X509_LOOKUP_by_issuer_serial
0001:000d30f9* _X509_LOOKUP_by_fingerprint
0001:000d314c* _X509_LOOKUP_by_alias
0001:000d3228* _X509_STORE_new
0001:000d33aa* _X509_STORE_free
0001:000d3471* _X509_STORE_add_lookup
0001:000d3515* _X509_STORE_get_by_subject
0001:000d3ae4* _X509_OBJECT_retrieve_by_subject
0001:000d390d* _X509_OBJECT_up_ref_count
0001:000d3657* _X509_STORE_add_cert
0001:000d3fc1* _X509_OBJECT_retrieve_match
0001:000d398a* _X509_OBJECT_free_contents
0001:000d37b2* _X509_STORE_add_crl
0001:000d3abb* _X509_OBJECT_idx_by_subject
0001:000d3b27  _X509_STORE_get1_certs
0001:000d3d79  _X509_STORE_get1_crls
0001:000d40cd  _X509_STORE_CTX_get1_issuer
0001:000d42ec* _X509_STORE_set_flags
0001:000d4309* _X509_STORE_set_depth
0001:000d432b* _X509_STORE_set_purpose
0001:000d4348* _X509_STORE_set_trust
0001:000d4365* _X509_STORE_set1_param
0001:000d4382* _X509_STORE_set_verify_cb
Module: U:\extras\lib\libcrypto.lib(o_time.obj)
0001:000d4390  _OPENSSL_gmtime
0001:000d43dd  _OPENSSL_gmtime_adj
Module: U:\extras\lib\libcrypto.lib(bio_enc.obj)
0001:000d48b7  _BIO_f_cipher
0001:000d51fa* _BIO_set_cipher
Module: U:\extras\lib\libcrypto.lib(pcy_data.obj)
0001:000d52e0  _policy_data_free
0001:000d5346  _policy_data_new
Module: U:\extras\lib\libcrypto.lib(pcy_map.obj)
0001:000d5470  _policy_cache_set_mapping
Module: U:\extras\lib\libcrypto.lib(a_bool.obj)
0001:000d5640* _i2d_ASN1_BOOLEAN
0001:000d56c5  _d2i_ASN1_BOOLEAN
Module: U:\extras\lib\libcrypto.lib(b_dump.obj)
0001:000d57a0* _BIO_dump_cb
0001:000d5803* _BIO_dump_indent_cb
0001:000d5bb9* _BIO_dump_fp
0001:000d5be2* _BIO_dump_indent_fp
0001:000d5c33* _BIO_dump
0001:000d5c5c  _BIO_dump_indent
Module: U:\extras\lib\libcrypto.lib(pk7_attr.obj)
0001:000d5c9b* _PKCS7_add_attrib_smimecap
0001:000d5d28* _PKCS7_get_smimecap
0001:000d5d90* _PKCS7_simple_smimecap
0001:000d5f07* _PKCS7_add_attrib_content_type
0001:000d5f64  _PKCS7_add0_attrib_signing_time
0001:000d5fe4  _PKCS7_add1_attrib_digest
Module: U:\extras\lib\libcrypto.lib(pem_oth.obj)
0001:000d606a  _PEM_ASN1_read_bio
Module: U:\extras\lib\libcrypto.lib(pem_lib.obj)
0001:000d6130* _PEM_version
0001:000d61ac* _PEM_def_callback
0001:000d62fa* _PEM_proc_type
0001:000d6393* _PEM_dek_info
0001:000d6480  _PEM_ASN1_read
0001:000d8317* _pem_check_suffix
0001:000d6927  _PEM_bytes_read_bio
0001:000d7b05* _PEM_read_bio
0001:000d72be* _PEM_get_EVP_CIPHER_INFO
0001:000d7084* _PEM_do_header
0001:000d6a8a  _PEM_ASN1_write
0001:000d6ba5  _PEM_ASN1_write_bio
0001:000d7771* _PEM_write_bio
0001:000d76a9* _PEM_write
0001:000d7a5a* _PEM_read
Module: U:\extras\lib\libcrypto.lib(bio_ndef.obj)
0001:000d83cb  _BIO_new_NDEF
Module: U:\extras\lib\libcrypto.lib(asn_mime.obj)
0001:000d88c3  _i2d_ASN1_bio_stream
0001:000d9c28* _SMIME_crlf_copy
0001:000d8aa8  _PEM_write_bio_ASN1_stream
0001:000d9081  _SMIME_write_ASN1
0001:000d96a8  _SMIME_read_ASN1
0001:000d9db0* _SMIME_text
Module: U:\extras\lib\libcrypto.lib(pcy_node.obj)
0001:000daa18  _policy_node_cmp_new
0001:000daa2d  _tree_find_sk
0001:000daa75  _level_find_node
0001:000daaef  _level_add_node
0001:000dac24  _policy_node_free
0001:000dac37  _policy_node_match
Module: U:\extras\lib\libcrypto.lib(pcy_lib.obj)
0001:000dacf0* _X509_policy_tree_level_count
0001:000dad08* _X509_policy_tree_get0_level
0001:000dad38* _X509_policy_tree_get0_policies
0001:000dad50  _X509_policy_tree_get0_user_policies
0001:000dad7d* _X509_policy_level_node_count
0001:000dadca* _X509_policy_level_get0_node
0001:000dae0f* _X509_policy_node_get0_policy
0001:000dae29* _X509_policy_node_get0_qualifiers
0001:000dae43* _X509_policy_node_get0_parent
Module: U:\extras\lib\libcrypto.lib(evp_key.obj)
0001:000dae60* _EVP_set_pw_prompt
0001:000dae99  _EVP_get_pw_prompt
0001:000daeb3* _EVP_read_pw_string
0001:000daee3  _EVP_read_pw_string_min
0001:000db006  _EVP_BytesToKey
Module: U:\extras\lib\libcrypto.lib(encode.obj)
0001:000db320  _EVP_EncodeInit
0001:000db377  _EVP_EncodeUpdate
0001:000db59e  _EVP_EncodeBlock
0001:000db539  _EVP_EncodeFinal
0001:000db6e2  _EVP_DecodeInit
0001:000db72f  _EVP_DecodeUpdate
0001:000db9d9  _EVP_DecodeBlock
0001:000dbb55  _EVP_DecodeFinal
Module: U:\extras\lib\libcrypto.lib(bio_asn1.obj)
0001:000dbbc5  _BIO_f_asn1
0001:000dc50b  _BIO_asn1_set_prefix
0001:000dc534* _BIO_asn1_get_prefix
0001:000dc55d  _BIO_asn1_set_suffix
0001:000dc586* _BIO_asn1_get_suffix
Module: U:\extras\lib\libcrypto.lib(bio_b64.obj)
0001:000dc5c0  _BIO_f_base64
Module: U:\extras\lib\libcrypto.lib(bf_buff.obj)
0001:000dd7e7  _BIO_f_buffer
Module: U:\extras\lib\libcrypto.lib(ui_lib.obj)
0001:000de5e0  _UI_new
0001:000de5fd* _UI_new_method
0001:000df634* _UI_get_default_method
0001:000de717  _UI_free
0001:000dea8e  _UI_add_input_string
0001:000deadc* _UI_dup_input_string
0001:000deb7e  _UI_add_verify_string
0001:000debcb* _UI_dup_verify_string
0001:000dec6c* _UI_add_input_boolean
0001:000decb9* _UI_dup_input_boolean
0001:000dee96* _UI_add_info_string
0001:000deee8* _UI_dup_info_string
0001:000def8e* _UI_add_error_string
0001:000defe0* _UI_dup_error_string
0001:000df08f* _UI_construct_prompt
0001:000df1fa* _UI_add_user_data
0001:000df217* _UI_get0_user_data
0001:000df222* _UI_get0_result
0001:000df8b9  _UI_get0_result_string
0001:000df329  _UI_process
0001:000df4d3* _UI_ctrl
0001:000df5af* _UI_get_ex_new_index
0001:000df5e6* _UI_set_ex_data
0001:000df60a* _UI_get_ex_data
0001:000df627* _UI_set_default_method
0001:000df654* _UI_get_method
0001:000df65e* _UI_set_method
0001:000df670* _UI_create_method
0001:000df6cb* _UI_destroy_method
0001:000df6f4* _UI_method_set_opener
0001:000df714* _UI_method_set_writer
0001:000df734* _UI_method_set_flusher
0001:000df754* _UI_method_set_reader
0001:000df774* _UI_method_set_closer
0001:000df794* _UI_method_set_prompt_constructor
0001:000df7b4* _UI_method_get_opener
0001:000df7cc* _UI_method_get_writer
0001:000df7e4* _UI_method_get_flusher
0001:000df7fc* _UI_method_get_reader
0001:000df814* _UI_method_get_closer
0001:000df82c* _UI_method_get_prompt_constructor
0001:000df844  _UI_get_string_type
0001:000df85b  _UI_get_input_flags
0001:000df873  _UI_get0_output_string
0001:000df88b  _UI_get0_action_string
0001:000df8e3  _UI_get0_test_string
0001:000df90c* _UI_get_result_minsize
0001:000df936* _UI_get_result_maxsize
0001:000df986  _UI_set_result
Module: U:\extras\lib\libcrypto.lib(ui_openssl.obj)
0001:000dfc7f  _UI_OpenSSL


                        +----------------------+
                        |   Imported Symbols   |
                        +----------------------+

Symbol                              Module
======                              ======

___libc_ForkRegisterModule          libc065
___init_dll                         libc065
___libc_Back_termDll                libc065
___libc_ForkDeregisterModule        libc065
__atfork_callback                   libc065
_PyLong_FromLong                    python27
_PyString_AsString                  python27
_PyOS_snprintf                      python27
_PyString_FromString                python27
_PyThread_free_lock                 python27
_PyObject_Free                      python27
__PyObject_New                      python27
_PyThread_acquire_lock              python27
_PyThread_release_lock              python27
_PyEval_SaveThread                  python27
_PyEval_RestoreThread               python27
__PyArg_ParseTuple_SizeT            python27
_PyBuffer_Release                   python27
__Py_NoneStruct                     python27
_PyThread_allocate_lock             python27
_PyString_FromStringAndSize         python27
_PyExc_ValueError                   python27
_PyErr_SetString                    python27
__PyArg_ParseTupleAndKeywords_SizeT python27
__PyArg_Parse_SizeT                 python27
_PyExc_TypeError                    python27
_PyType_Type                        python27
_PyType_Ready                       python27
_Py_InitModule4                     python27
__CRT_init                          libc065
__CRT_term                          libc065
___ctordtorInit1                    libc065
___ctordtorTerm1                    libc065
__errno                             libc065
___stderrp                          libc065
__std_memcpy                        libc065
___libc_GLocaleCtype                libc065
__std_memset                        libc065
___register_frame_table             gcc473
___deregister_frame                 gcc473
__std_memcmp                        libc065
__std_getpid                        libc065
__std_vfprintf                      libc065
__std_abort                         libc065
__std_strcmp                        libc065
__std_strlen                        libc065
__std_strerror                      libc065
__std_strncpy                       libc065
__std_strchr                        libc065
__std_malloc                        libc065
__std_realloc                       libc065
__std_free                          libc065
__std_strcpy                        libc065
__std_memchr                        libc065
__std_qsort                         libc065
__std_time                          libc065
__std_localtime                     libc065
__std_getenv                        libc065
__std_atoi                          libc065
__std_fwrite                        libc065
__std_fopen                         libc065
__std_fclose                        libc065
__std_fread                         libc065
__std_ferror                        libc065
__std_fseek                         libc065
__std_feof                          libc065
__std_ftell                         libc065
__std_fileno                        libc065
__std_setmode                       libc065
__std_fflush                        libc065
__std_fgets                         libc065
__std_strnicmp                      libc065
__std_strtol                        libc065
__std_strncmp                       libc065
__std_sscanf                        libc065
DosTmrQueryTime                     doscalls
DosQuerySysInfo                     doscalls
DosEnterCritSec                     doscalls
DosPerfSysCall                      doscalls
DosExitCritSec                      doscalls
DosAllocMem                         doscalls
DosQuerySysState                    doscalls
DosFreeMem                          doscalls
__std_strrchr                       libc065
__std_random                        libc065
__std_strcat                        libc065
__std_stricmp                       libc065
__std_strtoul                       libc065
__std_memmove                       libc065
__std_gmtime                        libc065
__std_fprintf                       libc065
___stdinp                           libc065
__std_fputs                         libc065
__std_fputc                         libc065
__std_tcgetattr                     libc065
__std_tcsetattr                     libc065
__std_sigaction                     libc065


                        +--------------------+
                        |   Libraries Used   |
                        +--------------------+

U:\extras\lib\libcrypto.lib
U:\tmp\ldconv_python2_7_dll_a_1a0352885a3d18b290.lib
U:\tmp\ldconv_libgcc_a_1a0352885a3d18ed28.lib
U:\tmp\ldconv_libgcc_so_d_a_1a0352885a3e1639c0.lib
U:\usr\lib\libc_alias.lib
U:\usr\local473\lib\libc_dll.lib
U:\usr\lib\libos2.lib
U:\usr\lib\libend.lib


                        +-----------------------+
                        |   Linker Statistics   |
                        +-----------------------+

Stack size:  0000 (0.)
Memory size:  000e4120 (934176.)
Link time: 00:00.22
